:020000041100E9
:103000007FB50023284C294D03932800217C284AB2
:1030100001F0DBFA002812D103232800217C03AA47
:1030200001F07AFA00280AD1224B039A9A4206D17B
:10303000214B2248E360224B636104B070BD02263D
:10304000217CFE2228001F4B009601F037FA002851
:1030500001D00020F1E71C4BA2899A42F9D1217CD2
:10306000FF222800194B009601F028FA0028F0D121
:10307000E389174A934203D1164B17486361DCE793
:10308000164A9342E5D1164B164A1B68934206D95D
:10309000C02304222800217C9B0001F078FA124B07
:1030A00012486361C9E7C0460862FF1F3C42FF1F28
:1030B000813700005959530059598320A0BE00118F
:1030C000FD4100111462FF1F595900001662FF1FD5
:1030D00083050000B141001180BE0011821500007F
:1030E0002C62FF1F87130000B942001190BE00112F
:1030F000002370B51A4E1B4C30006361637401F0FD
:103100008BF9402323744B2B0CD9CC233821AC22D0
:1031100030009B01217401F03AFA00280AD0002502
:1031200025740CE0FFF76CFF051E08D1237C0433E7
:10313000DBB2E7E70C4B0D4D63610D4BE381236878
:10314000002B08D1002D06D00C222900200008F009
:10315000DBFB2B7B6374300001F09CF970BDC04633
:103160003C42FF1F0862FF1F5142001170BE001158
:10317000AAAAFFFFF7B5164B0192C318021D002043
:10318000009388235B05D3181B685C1C1AD09CB283
:10319000402C18D88D781E0CAC466746CD782D0291
:1031A0003D43AE4206D1019800280ED110000C70AC
:1031B000240A4C7003249BB20733A343D218009B0C
:1031C0009A42DED3FEBD4432F9E71000FAE7C0466A
:1031D000FC0F0000802213B503000324019189B283
:1031E000520107319B18A14304305A1A88235B050A
:1031F000C3181B68591C03D190429241104016BD60
:1032000099B2402907D80B000733A343C018904256
:10321000ECD30020F3E74430F9E7134B134A1B6863
:10322000126810B5FA24934201D81A00F824104B02
:10323000E4021B689A4210D813000E4A12689A42A0
:103240000ED3013307D1F823DB029C4203D10A4994
:10325000054808F0A9FA200010BDFC24E402ECE7C0
:10326000FE24E402F7E7C04600C0071100D00711B2
:1032700000E0071100F00711FFFFFF7FF0B59BB0E2
:10328000150004900391402A00D9A0E006AB5980B4
:103290001A80FFF7C2FF0400042816D9002206A9ED
:1032A000FFF768FF052810D906AB1B88AB420CD18D
:1032B000002D07D0514B2A000499C01808F014FBC8
:1032C000002802D101201BB0F0BD06AB1D802000FC
:1032D0000699FFF77FFF041E7BD1069B0793FFF73C
:1032E0009CFF80235B01C618802307001B039E42BE
:1032F00001D3F826F60288235B05F31801931B68B7
:10330000013302D0019808F04FFC3D49019808F0C4
:103310004BFA3B1D0293331D05938822029B5205F5
:103320009B181B6808935A1C3CD044219AB2009108
:10333000402A04D80320D11D814389B2009103990A
:103340001B0C8B4224D0402A22D80122300008A92D
:10335000FFF710FF021E1BD1380008A9FFF70AFF74
:103360000400042831D9009A059B9B188022520141
:10337000B218934240D288235B05C118009A09A86D
:1033800008F0C2FA1D4B009A09A9F01808F06CFC6D
:10339000009A029B9446634402931A4B029AFB18CC
:1033A0009A42BAD388235B05FC1821680198013939
:1033B00008F0FAF9200008F0F7FB039A07AB5A80EF
:1033C00030000799FFF706FF0400002C03D100200E
:1033D00079E70428FBD988235B05E018069908F0F3
:1033E000E3F90323EA1C9A4300D16BE7034B0499EA
:1033F000E01808F039FC65E70424ECE7040000114C
:10340000FFFFFF7FF80F0000F7B505001400402A0A
:1034100021D8002701AE71803780FFF7FEFE042817
:1034200016D93A003100FFF7A5FE042810D93688D6
:10343000BC420BD0BD4209D0221CB44200D9321C80
:10344000064B92B2C118280008F05EFA30B2FEBDF9
:10345000C04300B2FBE703204042F8E7040000113C
:1034600037B5042204000D0001A81649FFF7CCFF70
:10347000020004280BD1019BA34208D3AB4204D025
:10348000104901A80195FFF7F9FE01203EBD0E4C41
:1034900023682000019308F087FB0199200001397F
:1034A000019108F081F980235B01E418074B9C42ED
:1034B000EED10422034901A80195FFF7DFFE0020A9
:1034C000E4E7C0465555000000C007110000081190
:1034D00030B589B008F020FB10226946254808F075
:1034E00023F9254B009A9A420ED1019B029A0F2B89
:1034F00033D8002101240698013B08D2002900D0CE
:103500000292029B013331D10023029325E0551C26
:10351000F2D102002100EFE710341022200004A9AC
:1035200008F002F9029B013301D1069B0293882324
:1035300004995B05C918059B06981A03120B0491A0
:103540000592814203D02B4201D108F0DDF9019BA5
:10355000013B0193019B002BDED1029B002B03D08A
:10356000049304984168084709B030BDE025014C38
:103570002D03EFE700000111504859368022F8B5BD
:10358000964C974BD200002120001C6008F004F9F3
:103590002300944A88331A60934B1A786A23002ACE
:1035A00000D01133E3620A232365904B37221B7846
:1035B0000820A3638E4B2118E361102323628D4BF7
:1035C0003B256361C823DB00A36123008C331A60B1
:1035D0002823013AE26320646364CA67043A211D28
:1035E000CA672100BC310D602100C0310860210094
:1035F000C4310B6021000635CC310D602100083D3F
:10360000C8310D602100D0310A602200D432106030
:103610002200D832136022000227E0322100176016
:103620004222DC310A6021001B3DE4310D602100A3
:10363000E83108602100EC310B6023000521F433F0
:1036400019602300F0331A602300183290331A6097
:1036500023009433186023001E3A98331A60AF2376
:10366000DB002360644BFA262363644B644DE36004
:10367000644BF031A3642300FF31FC33B600A1603A
:1036800021611E60A5627325E5656D3D6565A565D3
:1036900096255D4AAD00E264666258606766A5667D
:1036A00000270925A767E566584F594D6067200038
:1036B0002567E2673A6015279C30676007001A208B
:1036C00038602000A0300700212038602000A8309A
:1036D00007004C4838602000F83006602600642758
:1036E000A436376026005F3FAC3637602600033FC4
:1036F000B03637602600C637B4363760260000275C
:10370000B836376038269E60424E96205E64424E40
:103710005A66DE61414E9A645E62F53EFF3E9E62ED
:103720001E269A67354A8000DE661F675F67DD6583
:103730001D661862DA67BE23394A5B00E250394BD6
:10374000D838235004302250C4225200A350C6233C
:10375000E4205B00E1500433334AE1503349344BF9
:10376000D1603449800019503349E938FF38195085
:1037700032490430195032493248D161324911631B
:10378000324951631900F4310860CE2030494000BD
:1037900011603049195019002F48F83108602F493D
:1037A000D16582212E4A89005A501A002D490832CB
:1037B000D1671A002C49B432116088212B4A890044
:1037C0005A501A002A49883211602A4ADA6408F0ED
:1037D0005BFA012008F008F8F8BDC0460004FF1F9E
:1037E000AC64FF1F706FFF1F7844FF1F4A0AFF1F62
:1037F0003A07000080C3C9019A020000DC050000FE
:103800006A18000050C3000088130000F009FF1F71
:10381000204E00006509FF1F68100000C409000069
:1038200040420F0010270000FC00FF1FB51CFF1FC7
:103830000000FF1F092DFF1F9130FF1F292FFF1FC1
:103840007520FF1F6527FF1F9120FF1F3D22FF1FCF
:103850000120FF1F8929FF1F712AFF1F9119FF1FD8
:103860009528FF1FB925FF1FC525FF1F011FFF1F3B
:10387000B91FFF1F791EFF1F0223F0B50124604D01
:10388000604E2B70604B91B01C70604F0393336897
:1038900000212000FB7006F05DFE200006F054FDC4
:1038A0000023984205D0FA78552A02D0332A00D056
:1038B00099E03360042006F0B5FF08F055F8FFF7F3
:1038C0005DFE07F0C9FF1F2201240021504B10AEFE
:1038D0001A70504B1C70504B1970504B1968914323
:1038E000163A0A431A60602219689143403A0A4323
:1038F0001A6008F089F907F0CFFF494B9847C120BB
:10390000FF21484B80001A588A431A50C522920062
:1039100098588843BF390143995098584249084004
:103920008021C9010143802099509958C00509029E
:10393000090A0143995080213C48490108F0A4F844
:10394000032322003A49019400933A4808F0D4F93D
:103950002C22394905A807F0D7FF05AC61782078FB
:10396000023406F011FDA642F8D1344C344B2268E3
:1039700003201A40A023DB02134323608023226824
:103980009B041343236022682E4B1A4080239B0321
:10399000134323602C4A2D4B934200D8012007F09B
:1039A00073FF07F039FF80232268DB041343236091
:1039B000287808F0D9F8039B1878C0B207F0F4FF14
:1039C00008F0CAF82249042007F0E6FF06F0F6FEE8
:1039D00000F040F800F02EFE00F0DAFE00F016FADB
:1039E000002011B0F0BD00932100194A042007F017
:1039F000A3FE8023DB059C62FFF76AFD5AE7C04601
:103A00004A0AFF1F34F000407844FF1F3862FF1F4E
:103A1000480AFF1F490AFF1F680AFF1FBCF0004049
:103A2000E1A2000000E100E0FF00FFFF7C44FF1F77
:103A30000057FF1F7C54FF1F98BD001114F0004079
:103A4000FF7FF8FFFFFF9FFF0080FF1F706FFF1FCA
:103A50003B000108002210B51100112007F074FE90
:103A600010BD0000F8B500230926364F364C3B62E6
:103A7000E3681120B343E36008F0FEF8112008F07A
:103A80005BF8112008F058F94023226810251343F1
:103A9000236080236268DB02134363608023A26893
:103AA00002211343A360A368284A08201340A3609F
:103AB0008023A2689B0113430122A360236CAB43C4
:103AC0002364236C1343236480231B013B62226B1A
:103AD0001F4B1A402263626B1A406263A26B1A404A
:103AE000A263E26B1340E363E3681A4A1340E360A6
:103AF00006F04AFC0121082006F05AFD8023164AF0
:103B00005B00516C11200B43536407F0E5FEFD216F
:103B1000C720124B124A89005A50A36B80002B43D6
:103B2000A363E3680F4A3343E3600F4B1958114016
:103B3000802212020A431A50802292051A600B4B0F
:103B40005D63F8BD00F000403CF00040FFFFDFFF88
:103B5000EFFFEFFFFFFF7FFF003800400000FF1F77
:103B60005118FF1FFF00FFFF00E100E000000540CB
:103B7000E12010B5C00408F007F910BD70B52B4C5A
:103B8000238C002B2AD0FA22D200934201D2FFF7D5
:103B9000EFFF228A238C002A21D1DA00238263825C
:103BA000A382E38223836383A383E383226062602F
:103BB000A260E2601E4D1F4A6420EB8093420AD847
:103BC000FA220020D200934205D91B4A0A219818F4
:103BD00007F072FFC0B200232872238470BD072053
:103BE000E11CCA7F01320240CA7705D10325201D9E
:103BF000C17F01312940C17708325200A35200230E
:103C000021001A00088A01321B180231082AF9D152
:103C1000221DD27F9200A350626823689B18A2687D
:103C20009B18E2689B185B099BB2C3E77861FF1F92
:103C30002062FF1FB70B000030F8FFFF30B503A86C
:103C400004880B20002C0ED14968074D087849786C
:103C5000090201430A20A94205D10121200019804F
:103C6000024B1B7A137030BD192A00002062FF1F1F
:103C7000F7B5150008AA16884A680F4F14785278CD
:103C8000120222430A24BA4214D10122DBB2019269
:103C900000962A0007F0E2FC041E0BD1074B1B68BC
:103CA000002B07D068782A78000210434242504126
:103CB000013098472000FEBD02290000A461FF1FCB
:103CC00030B5012503790400BFB02B4211D00A4959
:103CD000408807F02FF828420BD0084B01A95B8DD4
:103CE0004D800B80064B00221B7A60880B7104F01C
:103CF00013F93FB030BDC0469C61FF1FB040FF1FAD
:103D00002062FF1F10B50549054806F0C9FF0421D0
:103D1000044A054806F086FF10BDC0469C61FF1F9F
:103D2000FFFF0000C4BD0011B040FF1F10B50248E6
:103D300004F074FF10BDC046C13C001101230370A4
:103D40000B4B1A7A4270022282709A78C270DA782B
:103D50000271032242711A7982715A79C2710C225E
:103D600002729A794272DB7983720B207047C046E7
:103D70002062FF1F022310B50370013B437005331F
:103D8000837010330371443B43712A33837144338E
:103D9000C37100230372064B04001B8843720A3070
:103DA000FFF7CCFF831D0A30C0B2E37010BDC046E0
:103DB0002062FF1F10B5142007F046FF124B14229B
:103DC0000021186007F0E8FC002007F025FE012024
:103DD00007F07AFF022007F0BFFD032004F0C2F9CC
:103DE000042006F0D7F9052003F000FC062004F0BB
:103DF000CDF8072001F0B0FA082006F0F3FE092004
:103E000001F08AF810BDC046A861FF1F07F0ACFFA3
:103E1000012007F019FE07F087FD0000094B10B5DF
:103E20000400984205D0012904D12000064906F07B
:103E300037FF10BD0229FCD1013904F0ADFE002886
:103E4000F3D0F6E7FEFF0000CE61FF1F70B50D7ADC
:103E5000100004AA2C00168810221440154220D10C
:103E6000002E20D10A78022A18D14A685178157894
:103E70000E4A09022943914205D00D4A914209D0C8
:103E80001C800A2404E014220A491A8007F03CFD31
:103E9000200070BD0C2208491A80F7E71C8001241D
:103EA000F6E70824F4E70B24F2E7C046F3FF00002E
:103EB000F4FF00000443FF1FBCBE001110B5040056
:103EC0000749084806F0ECFE074804F0E7FD00202B
:103ED000E40704D50721054A054806F0A3FE10BDF6
:103EE000CE61FF1FFFFF00001D3E001108BE001144
:103EF000F440FF1F00B50C4BBFB01A780B4902A865
:103F000000F000FD6B4680B2D880002809D06A46D8
:103F1000074B01A91B889380064B0022188803F0E9
:103F2000FBFF3FB000BDC046AC61FF1FAD61FF1F8E
:103F30004E41FF1F5842FF1F00B50C4BBFB01A780F
:103F40000B4902A801F02EFF6B4680B2D8800028F2
:103F500009D06A46074B01A95B8D9380064B00226E
:103F6000188803F0D9FF3FB000BDC046D661FF1FDF
:103F7000D761FF1FF440FF1F5842FF1FF7B50E0027
:103F8000377A1C0008AB11003D001A8820231D4021
:103F90001F423CD13378022B3BD173681F785B788A
:103FA0001B023B431E4FBB4208D01E4FBB4214D0E6
:103FB0001D4DAB4221D00A252800FEBD002A2AD182
:103FC000142C2AD82200F06807F09EFC174B1C70B6
:103FD000012CF1D9FFF7B0FFEEE7002A1BD1202C0E
:103FE0001BD82200F06807F08FFC114B04211C70D5
:103FF000104B187807F050FEDEE7E3B20124009280
:1040000001940A00310007F029FB0500D4E70825D8
:10401000D2E70125D0E70B25CEE70D25CCE7C0463A
:10402000F3FF0000F4FF000002290000D661FF1F2B
:10403000AC61FF1F5862FF1F332310B504000370EB
:104040000A220749013007F05FFC064B0F201B686E
:104050001A0AE37222731A0C1B0E6273A37310BD4B
:104060002062FF1F4862FF1F30B50125037904005D
:10407000BFB02B4213D00B49408806F05BFE2842AC
:104080000DD06A46084B02A81B889380FFF7D4FF27
:104090006B46D8800022608801A903F03DFF3FB045
:1040A00030BDC046CE61FF1F4E41FF1F10B5024814
:1040B00004F0B4FD10BDC0466940001170B5160093
:1040C00004AA148805AA15784A6850781178000265
:1040D0002A4A0843801805284BD807F015FD03131A
:1040E0001E29343F0720032C0BD80422121BAA429E
:1040F00000D92A0022491A803000091907F004FC6F
:10410000002070BD0720112CFBD81222121BAA42DE
:1041100000D92A001B491A80EEE707200E2CF0D8A0
:104120000F22121BAA4200D92A0017491A80E3E77E
:104130000720032CE5D80422121BAA4200D92A002A
:1041400012491A80D8E70720032CDAD80422121B60
:10415000AA4200D92A000E491A80CDE70720032C75
:10416000CFD80422121BAA4200D92A0009491A807A
:10417000C2E700220A201A80C3E7C046DCD5FFFF51
:1041800053BE0011F461FF1F43BE00113EBE00117B
:1041900039BE001134BE001110B50D21024A03488A
:1041A00006F040FD10BDC04628BE00116441FF1F4F
:1041B00013B5104C0423217C01AA00F0ADF90028AE
:1041C00015D16B469A88236852BA92B2534322891A
:1041D00009491B0C9B184B806B46DA88636852BAFE
:1041E00092B2534362891B0C9B188B8016BD012031
:1041F000FCE7C0460862FF1F2062FF1F13B5124C88
:1042000006236A46217C00F087F9002819D16B4605
:104210001988236849BA89B24B4321890B4A1B0C80
:104220005B1853806B46D97803335B781B020B43D2
:104230005BBA61689BB24B4361891B0C5B1893802E
:1042400016BD0120FCE7C0460862FF1F2062FF1F69
:1042500037B5174C07236A46217C00F05DF900282A
:1042600024D16B461B787F2B20D86B46DD78F0235A
:104270002A041B031A406B469B880E495BBA9BB20B
:104280001A4323682D09534322891B0C9B184B802A
:104290006B465A789B7812031B011A4363682A43C2
:1042A000534362891B0C9B188B803EBD0120FCE7A9
:1042B0000862FF1F2062FF1F7FB50226154C0022F7
:1042C000217C03AB0096050000F0F8F8002802D02E
:1042D000012004B070BD0E23217C0122280000962D
:1042E0006B4400F0EBF80028F2D16B469A89236802
:1042F000D2BA5343228908491B149B184B806B4642
:10430000DA89636852BA92B2534362891B0C9B18D4
:104310008B80DEE70862FF1F2062FF1F70B5184C1C
:10432000237C002B0FD0382B0ED1164D280000F027
:1043300073F8CC23AC222800217C9B0100F027F9E4
:10434000280000F0A7F870BDE3890F4A934209D115
:104350000C4D280000F060F800222800217C00F0BD
:1043600005F9EDE7094A9342EDD1064D280000F02A
:1043700053F890222800217C920100F026F9DFE713
:104380000862FF1F3C42FF1F8305000083200000DE
:1043900070B5144C237C002B1FD06369002B1CD0FC
:1043A000114D280000F038F8636928009847040090
:1043B000280000F06FF8002C10D10C4B0422995EFD
:1043C000002905DA9C801A8801321A80200070BD0D
:1043D000074A9142F7DD9A80F5E70124FEF788FE4F
:1043E000F4E7C0460862FF1F3C42FF1F2062FF1F28
:1043F0000F27000010B58024064AA4001168436B03
:10440000234205D113685B1A032BF8D9012010BD94
:104410000020FCE76008FF1F70B5C17905000C00A3
:10442000631E9C411A4BE402E41849000460C9B2BF
:10443000007906F0F3F8E979687949000131C9B2E9
:1044400006F0ECF8E8790930C0B207F075FC0023FB
:10445000E36661332360AA795B3B002A0ED02268B1
:104460009A43023B134323600A23E3610733236229
:1044700000232363A3630133E36370BD22689A437F
:10448000022313432360462363610633A361EFE7EE
:104490000050004070B5002504000368DD66C07957
:1044A0000930C0B207F0E8FB2900207906F052F885
:1044B0002900607906F04EF870BD0000F8B51E00C6
:1044C00006AB1D78002304681700E366616007F0FF
:1044D00023FB01238022E3662B0027615200013B6E
:1044E00008D207F0F9FB08200A4A1168002D03D111
:1044F0002800F8BD2261F2E7236F034203D023694D
:10450000013D3370013613685B1A032BEED9012588
:10451000EEE7C0466008FF1F70B51C000023056869
:104520001600EB66696007F0F7FA01238022EB665C
:1045300023005200013B08D207F0CEFB08200A4AB4
:104540001168002C03D1200070BD2A61F2E72B6FA7
:10455000034203D02B69013C3370013613685B1AA8
:10456000032BEED90124EEE76008FF1F002370B58E
:1045700004681500E366616007F0CEFA0123E36684
:10458000256107F0A9FB2000FFF734FF70BD70B56F
:104590001D00002304681600E366616007F0BCFAA2
:1045A0000123E36626610F33626B1A42FCD02B0AAB
:1045B00023611023626B1A42FCD0EDB2256107F033
:1045C0008BFB2000FFF716FF70BD002370B5046859
:1045D0001500E366616007F09FFA0123E3662B0A8A
:1045E00023611023626B1A42FCD0EDB2256107F003
:1045F00073FB2000FFF7FEFE70BD70B51E000023A8
:1046000005681400EB66696007F086FA0123A619B5
:10461000EB660F33B44205D107F05EFB2800FFF7CD
:10462000E9FE70BD21782961696B1942FCD0013423
:10463000F0E7000010B5084CE368002B08D1802299
:10464000064B52021B689B186360054B1B68236076
:1046500007F002FAA06010BD4862FF1FC8F00040DA
:10466000CCF0004070B5184A936A916A9942FBD128
:1046700016498A689A421FD39A1A8B60144B0126F6
:10468000186893B2D202D20E4343424300204C68D2
:104690001B0A1B1912029B180E4C0A684B60551C12
:1046A000A3420CD8002801D04B600A600A4A13606C
:1046B00008680A4B186070BD581E821ADDE7084A68
:1046C00030009B182A00EAE700F000404862FF1F14
:1046D000140AFF1F40420F00C8F00040CCF0004019
:1046E000C0BDF0FF70B5214C23793F2B01D93F238A
:1046F00023711F4B22791A701878C0B207F0F4F9B1
:1047000018231C491C4A0B801C4913800B805380C2
:10471000A3791B4980200B800C21938001334B43EC
:10472000184D191C0001834200D9011C2980D18039
:104730006379002B16D101336371237A012B01D8E1
:10474000022323726279237A0F4853430A21584384
:1047500007F0B2F90D4D2860E379052B01D810233D
:10476000E37170BDA02BE8D9A023E5E73C62FF1FF1
:10477000480AFF1F5642FF1F2444FF1F5442FF1FD9
:104780005242FF1F5042FF1F710200002C62FF1FA8
:10479000F8B520210020FEF763FE114C011E114DDB
:1047A00009D10C22104BC1CBC1C4280006F0F4FF84
:1047B000FFF798FFF8BD0C2220000C49FEF724FEFD
:1047C0000C2802D0084B43CB43C40C2228000849D4
:1047D000FEF71AFE0C28EBD00C220021E5E7C046BC
:1047E0003C62FF1F0862FF1FB0BE0011FC0C0000FE
:1047F000F50C0000F0B51D4C8022A5440400882073
:1048000069465201400507F0F7F9902212016A4407
:104810001300200032C832C316C816C38023144CBC
:10482000144FA6689B033343A3603B6006F0FCFF74
:104830008823A0685B05C01807F0B6F90025882317
:1048400029008022A0685B05C01840196944520005
:1048500007F00AFA80230135FF355B019D42EED156
:10486000A6603E60044B9D44F0BDC046FCEFFFFFD8
:104870009443FF1F9808FF1F04100000F0B50400C8
:1048800087B0002825D0684606F07EFF1B4C022822
:1048900006D106226946200007F026F8002816D027
:1048A0006946002301250F262F00E25C0133100921
:1048B0001030874038002F00324097403A000243C2
:1048C0004A610439062BEFD16846FFF793FF07B022
:1048D000F0BD182269460A4807F08EF96A46A3001F
:1048E000D358013305D01822FF21684606F054FF43
:1048F000EAE70134062CF1D1E9E7C0466509FF1F5C
:1049000000090011F0B5002504000E0085B0AA4290
:1049100000D186E04B1C087801934B788978377971
:1049200009021943F3783F061B040B431F43039707
:1049300020706570252800D196E033D8112813D84F
:1049400007F072F969003501350135013501AA001A
:10495000B800B100350135013501350135013501AA
:10496000350135010F012F01232800D1E8E0DB28B4
:1049700000D03EE1042A00D8B1E01025052A05D078
:10498000551F2A003800711D06F0BEFF05223100B8
:10499000200006F0B9FF2A003900601D06F0B4FFC0
:1049A00005353EE0562859D010D8332800D1A7E06D
:1049B000552839D02628DAD1A44B29001322180013
:1049C0001D0006F0E9FEFEF793FB5CE0712800D1C4
:1049D00077E0722800D189E0602800D195E0DC28DA
:1049E000C5D1022A00D87AE07378BFB26370B37879
:1049F000A370032A05D0033A390092B2F01CFEF7E7
:104A00003DFC10223900E01CFEF7FEFCC51C00280E
:104A100007DA607070E00C2220008D4906F074FF08
:104A20000C25280005B0F0BD013A8A4D0C2A13D898
:104A3000002A0AD02800019906F066FFFFF752FE0F
:104A40000C2228008449FEF719FC29000C22601C66
:104A500006F05AFF0D25E4E70C22EBE77D4D7F4B76
:104A60002A0043CB43C2E9E7013A784D0C2A11D81A
:104A7000002A08D00199280006F046FF0C222800E1
:104A80007749FEF7FBFB29001322601C06F03CFF70
:104A90001425C6E70C22EDE706227249601C06F0D9
:104AA00033FF0625BDE712226F49601C06F02CFF7C
:104AB0001325B6E708226D49601C06F025FF09257D
:104AC000AFE7012A0ED07178F02908D8684D288800
:104AD00001F0C4FD674B2A885200D35A00E0FF233F
:104AE000637009E0624A634B1288F5E7624B012A62
:104AF00004D072789A706270022592E79B78EFE793
:104B00002000FFF799FA05008BE7013A5A4B5B4DFD
:104B1000072A10D8002A10D00121280059700199C5
:104B200006F0F2FE01F05EF829000722601C06F094
:104B3000EBFE082575E70722EEE700225A70F3E73F
:104B4000042A04D94E4D2F6006F086FFA860FFF7B7
:104B500089FD0422039003A9601C06F0D5FE0525FB
:104B60005FE7484D062A15D906222800019906F06C
:104B7000BBFE00280ED006220199280006F0C4FED4
:104B8000062241492800FEF779FB01233A4A917831
:104B90000B43937029000622601C06F0B5FE072522
:104BA0003FE7012A9BD07078FFF768FEA4E7012851
:104BB00000D0DCE6931E354F132B06D87378002BFC
:104BC0000BD100F017F900F04DF9314B39001D7889
:104BD000601C6A1E06F098FE23E7551E2A00019904
:104BE000380006F091FE38002A49AAB2FEF746FBCB
:104BF000E9E7DA281DD1042A00D870E7082A15D978
:104C0000B37972791B021343F27912041A43337A8F
:104C10001B0613433B603B680522310020000393D1
:104C200006F072FE0422601D03A946E7FE236370AE
:104C3000F1E7DE2800D052E7511E012A01D10025FC
:104C4000EFE6019800F0B4FFF9E7C0460862FF1FE5
:104C5000BCBE00113C62FF1FFC0C0000B0BE001186
:104C6000F50C00001462FF1FF461FF1F9843FF1F43
:104C70005842FF1FB064FF1F3862FF1FF542FF1F3D
:104C80004862FF1F6509FF1FADAC00003964FF1FBC
:104C90003764FF1FAEDE000070477047020010B59A
:104CA000094B0A32094C92B2DA815A8298811882F1
:104CB000207802F039FB0422054B012120781A707C
:104CC00006F0EAFF10BDC0462243FF1F8264FF1FAB
:104CD0008164FF1F013870B5042809D806F014FF5D
:104CE000030928081200234B0221187806F0D4FF8C
:104CF00070BD204B0821187806F0EEFE00221E4BF6
:104D00001A72F5E7802200241B4B1A4D52001A81BB
:104D100008211A682878DC7206F036FF210028780E
:104D200006F04AFF012000F063FE00F05BFFDFE7C2
:104D3000104B0821187806F0CFFE1048FFF71AF83C
:104D40000F4B104A9B79002093800F4A13808022DA
:104D5000094B5200D8721A8100F04AFE00F042FF5F
:104D60000A4B9B78002BC3D0094A136006F044FE1F
:104D7000BEE7C0465862FF1F2C62FF1F6142FF1F43
:104D80003C62FF1F2444FF1F5242FF1F3862FF1F77
:104D900034F0004010B500290BD1012809D1054B92
:104DA0001B78002B05D02622034B04485A72FFF7CC
:104DB00075FF10BD5A64FF1F2C62FF1FC40900005D
:104DC0000300F0B50A4D8E18B14202D1520080188E
:104DD000F0BD0C782F6824093C5D0F271C700C78FF
:104DE00001313C402F683C5D5C700233ECE7C0460B
:104DF0004C42FF1F0D22124B10B51A700C23114CA0
:104E000011492370093A033B1048637006F07CFD9A
:104E10002D2301220E490F48A371FFF7D1FF012274
:104E20000D49FFF7CDFF01220C49FFF7C9FF030031
:104E300000200B4902001870FEF720FA10BDC04692
:104E40005664FF1F3764FF1F53BE00113964FF1FF4
:104E50006709FF1F3E64FF1F6609FF1F6509FF1FEB
:104E6000AEDE000070B5134C142220001249FEF78C
:104E7000CBFA431E114D132B19D8AB78002B16D04B
:104E8000431C2B7009236B700023001903702878D2
:104E90000B4B01302900C0B2187006F09DFE297836
:104EA00022000139C9B2002005F0DAFD70BDFFF71C
:104EB000A1FFECE73964FF1FAEDE00003764FF1F7F
:104EC0005664FF1F10B5114B1A781870002A0ED0C7
:104ED00000280BD10E4B1A78062A07D85423D3404A
:104EE000DB0703D50B4B187802F01EFA10BD002823
:104EF000FCD0074B1B78012B02D0033B022BF5D8CB
:104F0000044B0121187806F0C7FEEFE75A64FF1F33
:104F10008164FF1F8264FF1F70B54A4E4A4A4B49A5
:104F20003070012005F028FC00F0DAFEFEF7E0F812
:104F300006F0A2FC032246494648FFF741FF2D2414
:104F4000030004221C7044490130FFF739FF30236D
:104F50000470424D424C437083702E3B0622200069
:104F60004049EB87FEF750FA062813D0200006F0E0
:104F70000BFC022809D00321200006F0CDFE8D2372
:104F8000E3706E3B237119336371062220003549AB
:104F9000FEF774F9344B1B68FC335C64FFF762FF67
:104FA0000020FFF78FFF314C314A0121314B12783D
:104FB000207802F07BF9304A304B127800212078BB
:104FC00002F074F901222E4B1A702E4BDB78552B10
:104FD00031D12D4B3B325A722C4B2D4AAB81EA8199
:104FE0002B826A822021307806F03EFD012040426B
:104FF00005F082FD0120404205F01EFEFFF7CCF8CF
:10500000FEF780FE00F0B2FC01204042FEF756FFA2
:10501000012006F021FEF02001F004FB0121307890
:1050200006F03AFE307802F0DBFA1A4806F0FCFC93
:10503000FEF718FD70BD6422174B5B7953431A00CD
:105040000A32CBE75862FF1F954D0011994C0011B1
:105050009843FF1FF461FF1F1462FF1F2243FF1FCD
:105060006509FF1FADAC0000AC64FF1F8264FF1F29
:105070008042FF1F6142FF1F5664FF1F3764FF1FFE
:105080002864FF1F3862FF1F2C62FF1FC409000045
:10509000CE0900005A62FF1F3C62FF1FF8B50A00EC
:1050A00020230D001A40194263D05E4B1B78002B61
:1050B0005CD0FFF7D7FA5C4B5C4C5D4E9968626838
:1050C000737A8A1ADB039A4202D36160FEF7CAFC44
:1050D000327A217A531EDBB2994205D1FFF71EF9CD
:1050E000002000F0B5FD15E09142F9D300272772AA
:1050F000FFF74EF9A37ABB4202D0A772FEF73EFD3E
:10510000012000F0A5FD4B4F3800FEF733FE3900BB
:1051100006F0CAFD637A002B25D0013BDBB2637237
:10512000002B20D1444BDB78552B01D106F064FCD9
:10513000E37A002B12D00023A27AE3729A4202D0C3
:10514000A372FEF71BFD3D4A3A4F13883800013326
:105150001380FEF70FFE390006F0A6FD6423707978
:105160005843FFF79BFD237A0133237220206840C8
:10517000F8BD0BB2002B0ADA314B187806F0FCFDB3
:10518000002801D006F040FB80200002EFE7022457
:10519000214206D0254B01201A72FFF793FE200012
:1051A000E5E70B071ED5FFF75DFA1F4B1F49204CA3
:1051B00098684A68637A821ADB039A4202D348608D
:1051C000FEF750FCFFF7E4F8FFF7A8F8012000F025
:1051D0003FFD00F0E5FB2368DB0701D5FEF766FF26
:1051E0000820C4E7CB0609D5FEF7C8FC0D4B1B7899
:1051F000002B01D1FEF79AFD1020B8E701242142CF
:1052000007D0104800F06CF806F06EFD00F006FDC7
:10521000C5E70424080020402142A9D0FEF76AFE19
:10522000BDE7C0465A64FF1F4862FF1F2C62FF1F84
:105230003C62FF1F6142FF1F3862FF1F2062FF1F99
:105240005862FF1F4442FF1FF0B51B4B1B4F1B88CA
:105250003A8804001A4E1B4D85B09A420DD8328808
:105260009A420AD3184B1A882B889A4205D1174ABA
:10527000174B12881B889A421BD0052001F028FA90
:105280003B8802AA13803388019053802B88114DEC
:1052900093800F4B02A91B88D3800F4B2A78188864
:1052A00002F044FF0D4B08212878019A1C7006F08B
:1052B00093FB05B0F0BDC0462664FF1F5642FF1F9A
:1052C0005442FF1F5242FF1F2464FF1F2264FF1F2E
:1052D0005042FF1F8264FF1F5842FF1F2064FF1FC0
:1052E00013B50C4B1C78002C11D1002801D00A4BAF
:1052F00018600A4A0A4B11780A4A10780A4A019241
:105300000A4A0092002205F0A3FA200016BD1124DB
:10531000FBE7C0468164FF1F1C64FF1F8064FF1F02
:105320007064FF1F8264FF1F5C64FF1F6064FF1FC7
:1053300010B5064B12201B78052B06D1044B132207
:105340001988044B187801F09FFB10BD8164FF1F82
:105350005842FF1F8264FF1F10B500240122114B29
:1053600052421870104B1C70104B1A8002F038F922
:1053700004220F4B21001A700E480C3206F0FCFB81
:10538000102221000C4806F0F7FB07220B4B1C6093
:105390000B4B1C700B4B1C700B4B1A700B4B1C7087
:1053A00010BDC0468264FF1F8164FF1F5842FF1F6B
:1053B0008064FF1F7064FF1F6064FF1F5C64FF1F39
:1053C0003664FF1F3564FF1F5A42FF1F3464FF1FFE
:1053D000F8B5174C0600257806A814240078052D8A
:1053E00023D1B41F134FA5B21824BD421DD88D1F61
:1053F000ADB2BD4219D8FA256D00AA4215D21D00E2
:105400000D4F0A3DADB2BD420FD80C4C26800C4C5E
:1054100021800C4900240A800B4A1380FFF714FFF7
:105420000A4B0421187806F057FB2000F8BDC0464F
:105430008164FF1F790C0000750C00005642FF1FAD
:105440005442FF1F5242FF1F5042FF1F8264FF1F42
:10545000F0B50BB20D0089B0002B00DB70E1A44E5B
:10546000307806F089FC041E50D00378A22B00D1BE
:1054700022E1D02B1AD0912B45D143780E2B42D16B
:105480009C4B82889A423ED19B4A83681278052AB7
:1054900039D1032018567F2835D0984B1B68002B34
:1054A00031D05B68002B2ED098472CE080780728FD
:1054B00029D806F029FB0428183F3F74A8D8637840
:1054C000002B0CD101218C4B19708D4B1A78002ABE
:1054D0005BD08C4B307801F0E9FE002855D00722D4
:1054E000854B1A7051E061780029F8D1E378002BE0
:1054F00011D0854A854B1278307801F0D7FE607064
:105500006378002BEBD1200006F07EF980200002AA
:10551000684009B0F0BD784B1B78022BF3D0012115
:10552000307806F0D1FA0028EAD10121307806F06F
:10553000B3FBE5E76378002BD1D16F4F032807D188
:105540003B78052B02D101333B701EE00223FBE7C1
:105550006F4B1A886F4B0293002A0BD01B78002BDD
:1055600003D00121307806F037FA3B78062B04D1BE
:10557000013BE9E7029B1A70F7E7042B41D10121B7
:10558000029B3078197006F087FB5C4B1B68002B80
:10559000B9D01B68002BB6D0574A107884E76378DF
:1055A000554F002B27D10622211D5B4806F0ACF990
:1055B00062895A4B5A491A80A2895A4B1A80E38948
:1055C0000B800521397058490A80584A1380228A75
:1055D000574B1A80574B1B78012B09D11F2001F024
:1055E00077F8FA22920042430421307806F0F4F969
:1055F0000022484B75E7312B00D070E70022454B65
:105600001A700323A0E706220021434806F0B4FAEB
:105610000023454A04211380444A30781380444AC9
:10562000138006F059FA0821307806F055FAA3796C
:10563000083B5A425341304A03331370304B1B78B6
:10564000002B06D0334B30781A78002A06D001F0B0
:105650006BFE0122314B52421A8096E701211970EC
:1056600006F01AFBF5E70821307806F035FA637882
:10567000002B00D047E72C4B2D4F0293E388029A72
:1056800004211380294B307803932389039A1380D4
:1056900063893B8006F018FA002800D033E7264BD8
:1056A0001B68002B00D12EE7039902983A880988DD
:1056B00000881B68984726E74379132B00D022E720
:1056C0000389012B0AD11D4B1B78022B06D108211F
:1056D000307806F001FAFFF72BFE14E7052000F002
:1056E000F7FF08210200307806F076F90BE7C04694
:1056F0008264FF1F051400008164FF1F1C64FF1FEC
:105700008042FF1F6142FF1F5664FF1F3764FF1F67
:105710005864FF1F5A64FF1F2964FF1F5842FF1F70
:105720003064FF1F3264FF1F2664FF1F2464FF1FC5
:105730002264FF1F2864FF1F1864FF1F2064FF1FDF
:105740008020C001014200D0E2E6CB0731D5324BC8
:105750001B78002B1DD0314E05AC3378052B1AD1A8
:10576000023B23702E4B21001B7823722D4B1B789C
:1057700063722D4B187801F03DFD002809D00720F9
:105780002A4B30701B68002B03D01B68002B00D005
:1057900098470120BCE60E20254B06221B782549A0
:1057A0002370254B1B78637002ABC01806F0ACF871
:1057B000D8E7022308001840194209D0174B1B787C
:1057C000052B03D11D4B188806F026FA02209FE610
:1057D0000424214203D0FFF737FD200098E6082378
:1057E00008001840194200D193E6154B1C78012C93
:1057F00003D0022C0DD008208AE6124B124A13491E
:1058000013481B881288098800880094FFF7E0FD80
:10581000F1E7FFF78DFDEEE75A64FF1F8164FF1F7C
:105820005A42FF1F3464FF1F8264FF1F1C64FF1F66
:105830003664FF1F5B42FF1F3564FF1F5842FF1F86
:105840002064FF1F5042FF1F5242FF1F5442FF1FA0
:105850005642FF1F10B502A804880B20002C10D15F
:10586000496808784978090201430C48814209D106
:10587000022119800A4B59881170DB7800205BB235
:10588000537010BD074C0A20A142FAD102211980A1
:10589000034B998811705B79F0E7C0466E2A0000CF
:1058A0002062FF1F6F2A0000F7B5150008AA1688AE
:1058B0004A680F4F14785278120222430A24BA42DF
:1058C00014D10122DBB2019200962A0005F0C6FE37
:1058D000041E0BD1074B1B68002B07D068782A7871
:1058E0000002104342425041013098472000FEBD63
:1058F000022900009464FF1F30B5012503790400DC
:10590000BFB02B4225D01449408805F013FA284235
:105910000CD0124B01A95B8D00220B8002234B801F
:105920000F4B5B888B80608802F0F6FA0D49608827
:1059300005F000FAC0070CD50B4B01A91B8800220B
:105940000B8002234B80064B9B888B80608802F083
:10595000E3FA3FB030BDC0468C64FF1F8442FF1F96
:105960002062FF1F8464FF1FDE42FF1F10B5074C3B
:105970000749200005F094F92000064905F090F948
:105980000721054A054805F04DF910BDFFFF00004D
:105990008C64FF1F8464FF1FDCBE00118442FF1F64
:1059A00010B5024803F03AF910BDC046F95800118D
:1059B0000221430888400B400A31084003430E206F
:1059C000024AD17881430B43D3707047F542FF1FE1
:1059D000064A1379410705D580210B4380011371D5
:1059E000907170477F210B40F8E7C046F542FF1FDA
:1059F000054A5378002803D080210B435370704729
:105A00007F210B40FAE7C046F542FF1F0F21114BE3
:105A1000DA780A40DA70502810D901310A43DA7076
:105A20002022D9780A43DA704022D9780A43DA7002
:105A30008022D97852420A43DA7005E03C28EFD838
:105A40002828F1D81428F3D80122D9780A43DA702B
:105A50007047C046F542FF1FF8B57F23324D040062
:105A60006E789E43314B984205DD76232B70363B92
:105A700033436B70F8BD2E4B984203DA58232B70DA
:105A80001433F5E783B21A0000215F32294892B23D
:105A9000294F297082422DD9A9708C4203DA5B42CA
:105AA0001CB220232B70053420B20A2106F004F822
:105AB00004B2FA239B009C4233DB80232A785B42AA
:105AC00013432B706421200005F0F6FF0A2100B279
:105AD00005F012FF09B22A787B5C13432B700A2170
:105AE000200005F0E9FF0A2100B205F005FF09B228
:105AF0007B5C0AE08022AA70002CDADA5B421CB2DE
:105B000020232B705F23092CE9DC1E430A2120008F
:105B10006E7005F0F1FE09B2AA787B5C1343AB709E
:105B2000A8E7632CCEDCEDE7F542FF1F1B4E00001B
:105B30001DFCFFFF2A08000006BF00117F23F7B5F8
:105B4000194FCD013E7904009E433E71EDB26328AA
:105B500006DD093B33433B7140231D437D71F7BD97
:105B60000300093304DA582333433B716C23F4E711
:105B70000E4B019300280BDA0423444224B23B71FC
:105B80000A21200005F0B8FE019B09B25B5CE4E746
:105B90000928F5DD0A2105F08FFF019B00B21B5C8F
:105BA0001E433E71ECE7C046F542FF1F06BF0011E1
:105BB000F8B50A4F05003B780E00002B0CD0084CBE
:105BC0002000FEF729FC33002A0020003978FEF778
:105BD00014FD2000FEF75EFCF8BDC046A064FF1F68
:105BE000FC42FF1F70B50A4E0A4D07223100280003
:105BF00005F07AFE002809D0074C31000722280062
:105C000005F082FE08212000FFF7D2FF70BDC046DC
:105C1000F542FF1F9964FF1F9864FF1F7F2210B594
:105C20000A4B59789143033A1A70103A0A435A7052
:105C300078220E219A70DA788A43DA706B221A7110
:105C40000C3A5A71FFF7CEFF10BDC046F542FF1F58
:105C500010B5002832D01E4C0223E05E1D4B1B689D
:105C60005B062CD509233221584305F025FF41302E
:105C7000FF3000B2FFF7F0FE0520FFF799FE042287
:105C8000A35E154A6320934205DC32331800642179
:105C900005F012FF00B20121FFF750FF207AFFF755
:105CA000B5FE0020FFF794FE0C4B187805384342F0
:105CB0005841C0B2FFF79CFEFFF794FF10BD0A21C8
:105CC000053005F0F9FE00B2FFF7C6FE0320D4E769
:105CD0002062FF1F3C62FF1FDD2600008164FF1F62
:105CE00070B50024094D2800AC71FEF795FB102318
:105CF0003E212800064AFEF780FCA04200D13E3437
:105D0000044B28001C70FEF7C5FB70BDFC42FF1F52
:105D1000F6BE0011A064FF1F0200F0B501270A487B
:105D20000A4E51188B1A002B00DCF0BD08241578A0
:105D30004308684038404000805B013C58406D0893
:105D4000002CF5D10132EDE7FFFF000016BF001176
:105D5000F0B500250F269D4200DBF0BD4C5D070924
:105D600044403440A400A05801357840F3E70000D7
:105D7000F0B589B06A460D000B000F2711001035F1
:105D80001C780133260024093E40167054700232FC
:105D9000AB42F5D12023024AFFF7DAFF09B0F0BD8C
:105DA0001CBF0011F0B54E780B7889B036020C009C
:105DB000170001901E43012A61D9954B9E4200D8DD
:105DC00077E001339E421CD1062A17D1CA788B781E
:105DD00012021A430B791B0413434A7912061A4321
:105DE0008C4B5A6100221A705A808B4A5A608B4A37
:105DF0009A608B4ADA60002009B0F0BD8822520513
:105E0000EEE7884B9E423CD182498B78002B00D034
:105E1000F6E00C2A31D10F22A3789343E2781202E4
:105E200013432279120413436279120613434B6021
:105E3000E279A07912020243207A00041043627AC8
:105E400012060243CA60E27AA07A1202024376483E
:105E50004A81834208D804236E49142201980B70AA
:105E600005F052FD1420C7E71201D21889235B0503
:105E70009A42F0D801238B70BDE7022AFAD005239D
:105E8000EAE76A4A01239642E6D1FFF751FA052F65
:105E90000CD9E378A2781B021343227912041A4327
:105EA00063791B061343624A0393136005F0A4FD54
:105EB000A1E7584D2B78002B9DD1AB78002B00D15A
:105EC000A0E02B8901339BB20093B34200D091E054
:105ED000132AD4D9CF7C8B7C3F02122120001F4390
:105EE000FFF71AFF874200D08EE0002E3DD1E37805
:105EF000A2781B0213432279E96812041A436379DA
:105F00001B06134303930A228B4212D1FF23A37073
:105F1000E370237163716B89002B09D1E37B227CD1
:105F20001B0212041343A27B13431B0901336B8131
:105F300000226B89002B8ED0002A67D16868370158
:105F40003818000B6B6900030390984205D968610B
:105F500005F02AFEEB780133EB7068681022A11C73
:105F6000381805F081FE2E8145E76F89009A7B1E67
:105F70009BB293423AD1E278A37812021A43237972
:105F800005A81B04134362796C6812061A43EB6878
:105F900000920392211D0C22049305F0B5FC012010
:105FA000260004A940421036FFF7E2FE013F012F10
:105FB00017D1009A0B232861824200D04CE70422BB
:105FC0001C49200005F050FE042203A9686805F072
:105FD00013FEE968039AFF23914200D13CE7F73BA7
:105FE0003AE73100FFF7C4FE1036DFE70923B74276
:105FF000A4D831E7009BB34200D9FCE607232BE786
:10600000022329E7032327E7062325E70A2323E7BB
:10601000FFFE00000443FF1F00000111FFFF00000E
:106020005048593601FF0000FFFF001102FF000039
:1060300034F000401043FF1F10B5034C0B00012249
:10604000210000F06BFA10BDF96100110B8870B5EA
:1060500006000D000224162B11D92B00032209493A
:1060600000F05CFA041E0AD1074B2A881B88191C11
:10607000934200D9111C300089B200F0EFFA2000E1
:1060800070BDC04625620011B264FF1F10B54A788A
:106090000400013A0B000220012A07D80A78002ADE
:1060A00004D005222000024900F038FA10BDC04695
:1060B000536200110A7810B50B0004000220002A78
:1060C00004D007222000024900F028FA10BDC04683
:1060D000FF6200110A7810B50B0004000220002AAC
:1060E00004D009222000024900F018FA10BDC04671
:1060F0006563001110B5034C0B000B22210000F06A
:106100000DFA10BD9563001110B5034C0B000D2264
:10611000210000F003FA10BD0764001110B5034C14
:106120000B000F22210000F0F9F910BD616400118D
:106130000A7810B50B0004000220002A04D01122B6
:106140002000024900F0EAF910BDC0467164001158
:10615000002310B51322190000F0E0F910BD000073
:1061600010B5034C0B001722210000F0D7F910BD29
:10617000C3640011002310B51922190000F0CEF9F4
:1061800010BD000010B5034C0B001B22210000F0D5
:10619000C5F910BDFD640011F7B584890D00060036
:1061A0000121002C22D000238268D3561778002BBF
:1061B0001EDA0C2C1AD90C3CA4B213194088009397
:1061C000230002F086FE431E984101307B06DB0F60
:1061D0006B703F23013C1F40A4B22870AF70AC80AD
:1061E000002C07D0B3680133AB6000210800FEBD6E
:1061F0000020EBE7AC60F8E70B7803704B88437046
:106200004B881B0A83700B79C370042070470420ED
:10621000022B06D10020537811781B02009A0B4301
:10622000138070470B8803700B881B0A4370022091
:1062300070470420009983420AD1537810781B02DA
:1062400003430B80D37890781B02034300204B80DC
:106250007047F8B50D004B7801240021461C0370EF
:106260002B788B4201D82000F8BD6B78B01C4F1CF6
:10627000012B10D1890069184B88022233704B889A
:10628000B9001B0A7370691805F05EFC043604340B
:10629000A4B2F9B2E4E7122359436B185A880431C7
:1062A00032705B8810221B0A7370691805F04CFC71
:1062B00012361234ECE770B5049D14001E00052B55
:1062C00001D8042070BD637812781B0213432B8021
:1062D000E378A2781B02134302226B802A71211DEE
:1062E000681D063E05F030FCB2B22A81E92AE8D8E2
:1062F0002800A11D0A3005F027FC0020E2E700235A
:1063000010B50A789A4201D8900010BD9A008A18F8
:106310005488013304705488DBB2240A4470948892
:1063200084709288120AC2700430EAE710B5110036
:10633000029C062B04D004201022142B01D010BD87
:10634000022222714B7808781B0203432380CB780A
:1063500088781B02034363800431601D05F0F4FB61
:106360000020ECE710B50C788B7804315C43E4B284
:1063700003702200013005F0E7FB601C10BD042013
:10638000022B06D10020537811781B02009A0B4390
:106390001380704710B50C000A88023105F0D4FB59
:1063A000208810BD70B504000D0004981100012B69
:1063B00001D8042070BD1678527812023243028050
:1063C0000200F13255701470E125002C00D10C351B
:1063D000023B9AB24280AA42EBD80231043005F067
:1063E000B3FB0020E6E70420009983420AD15378EA
:1063F00010781B0203430B80D37890781B02034371
:1064000000204B80704710B50C000A88023105F05F
:106410009BFB208810BD000070B501211E000420E8
:10642000049C0E400B4218D1CB40DDB28D4214D9F2
:106430000A49DBB2098899420FD32300EE331D705D
:106440003300580011184978165C090231430133B2
:106450002152D9B28D42F4D8002070BD1C43FF1FD9
:1064600010B50C000A88023105F06EFB208810BDC3
:1064700010B50C788B7804315C43E4B203702200D1
:10648000013005F061FB601C10BD10B511000298D1
:10649000032B01D8042010BD14785278043B12025B
:1064A00022430280CA788C781202224342809AB238
:1064B0008280EB2AEED80431063005F045FB00203F
:1064C000E9E710B50C000B8803700B881B0A4370BA
:1064D0004B8883704B881B0AC3708A88043006314E
:1064E00005F032FBA088043080B210BD0420012BDF
:1064F00003D100201378009A1370704710B50C0078
:106500000B8803700B881B0A43704A8802300431E1
:1065100005F01AFB6088023080B210BDF0B589B07A
:1065200003931E4B029242000700D05A019102F0E1
:1065300020F81325061E2DD0029B01240370019B19
:10654000002B04D0001903999847001984B26B46B8
:106550001B7A5BB2002B0FDA1021380002F01CFB13
:106560001925002813D130003219E1B202F066FC7F
:10657000051E0CD10C34A4B2042304AA380005A9CA
:1065800093800696948101F0AFFD051E02D0300085
:1065900005F02AFA280009B0F0BDC046B064FF1F1C
:1065A00070B505000C0000280CD00020814209D0F5
:1065B00010222000044905F0C7FA01202B7823732C
:1065C0006B78637370BDC0465CBF0011F0B5060008
:1065D0000D0017001C0085B002291BD000201029D7
:1065E00007D1022B07D0102B03D115E00020102C6F
:1065F00008D005B0F0BD69463800FFF7D1FF2A008A
:1066000069460BE069463000FFF7CAFF2200694681
:10661000380004E0022BE9D12A003900300005F0EF
:106620004BFBE6E7031CF02800D9F02303200849C0
:106630009AB2013A0B80D317034006499B189B106E
:106640000B80D30F04499B185B100B807047C0462A
:106650002043FF1F1E43FF1F1C43FF1F034B1B88CC
:106660008B4202D3024B4000C15270472043FF1FB0
:10667000B064FF1F014B4000185A7047B064FF1F01
:106680001722014B1A807047B064FF1F70B50500D8
:106690000E2005F061FB041E13D0D02303700023ED
:1066A0000622837007494570033005F04DFA064B0A
:1066B0002100DA8A62811B7E2373044B187805F06F
:1066C00033FB70BDCC64FF1FBC64FF1F7043FF1F12
:1066D000262803D8024B4000C05A70470148FCE707
:1066E0002243FF1FFFFF000070B506000C00094D9C
:1066F0001C220021280005F03FFA074B1E70074BB3
:106700001C7005F041F90123002801D0002312205C
:106710002B7070BDBC64FF1F7043FF1FDD64FF1F43
:1067200070B505000D4C0800E260A1601022002148
:10673000656005F001F9012803D11021A06802F07D
:1067400058FD10220021280005F0F6F8012803D199
:106750001021606802F04DFD70BDC046BC64FF1F93
:1067600070B5041E05D1002903D006220D4805F09E
:10677000EBF90D4B1D78012D11D1002C05D1022212
:106780001A7005F0F9F8280070BD00221A70074B46
:106790001B78FF2BF7D02000FFF778FFF3E70025E9
:1067A000F1E7C046CC64FF1FBC64FF1F7043FF1FAE
:1067B000030010B5002801D1002010BD00780B4A5D
:1067C000002803D15988D1821B7913761378022BC4
:1067D000F2D10023984200D103331370044B1B788D
:1067E000FF2B01D0FFF752FF0120E6E7BC64FF1F3B
:1067F0007043FF1F002911D000280CD04B790128CD
:1068000003D140225242134303E03F2213400328A6
:1068100002D001204B7170474022F4E70800FAE7EC
:1068200070B5094D0100287800280BD0074C0622CE
:10683000200005F089F921002878FFF7DBFF200010
:1068400004F0BAFF70BDC046DC64FF1FB664FF1FD2
:1068500000290AD0012808D13F224B799343C02B4D
:1068600003D0403B5A425341981C704770B5174DB6
:1068700006002B78FF2B15D00A2005F06DFA041EB8
:1068800010D0D0230370C83B8370114B11491B7883
:106890004670C3700622043005F056F921002878AE
:1068A00005F042FA0C4B1B78012B0DD10B4B1B68EA
:1068B000002B03D09B68002B00D09847084B042185
:1068C0001878084A05F060F970BDC0467043FF1F94
:1068D000DC64FF1FB664FF1FD864FF1F0465FF1F41
:1068E0000865FF1F60EA0000014B98687047C046CA
:1068F000BC64FF1F014BDB6818687047BC64FF1F56
:10690000074B10B5DA68136801331360054B18782C
:10691000FF2803D08021C90105F0BEF910BDC04693
:10692000BC64FF1F7043FF1FF7B50E0002F0C8F8EC
:10693000051E1CD00E4B06621F78002F00D1077871
:10694000AB791020019305F007FA041E0FD0D02375
:106950000380C73B8370019BE91DC370062204308E
:1069600005F0F2F821003800E66005F0DDF9F7BD2A
:106970006E43FF1F014B18787047C046DC64FF1F51
:10698000054B002805D1054B1A78054B002A00D18C
:10699000014B18007047C046CC64FF1FDC64FF1F2A
:1069A000B664FF1F014B58687047C046BC64FF1FA8
:1069B000024B1868431E9841C0B27047E064FF1F45
:1069C000421E03000120152A03D9FF3B5A425341BE
:1069D000D8B27047F0B51C0000230E0085B00390BC
:1069E00002920B70029A934201D3002019E0E55CF9
:1069F0005A1CD2B2002DF8D0029851198142F4DC11
:106A00000233DFB2A35C18000193FFF7D9FF00281F
:106A100007D0013D019A0399EBB233708A4202D14B
:106A2000E01905B0F0BDDB19DBB2DBE710B50C00F7
:106A300002F09EF803001220002B03D0210058889A
:106A400004F0FAFE10BD000070B50E4D84006359CD
:106A5000002B15D0186A002801D004F07DFE2B59B8
:106A6000586A002801D004F077FE2B59986A002854
:106A700001D004F071FE285904F06EFE00232B5162
:106A800070BDC046EC64FF1F1C4B70B504000E00C7
:106A9000150099420AD11A4B1B68002B01D1122014
:106AA00070BD1B68002BFAD09847F9E7154B994247
:106AB00015D1134B1B68002B0AD01B68002B07D085
:106AC0009847002804D1104B1C70104B1D70E7E74D
:106AD00029002000FFF7AAFF0028E1D1F3E7080012
:106AE00001F0EEFF0028DAD003780320A342D7D1CB
:106AF0002900300004F0A0FED2E7C046FEFF0000EF
:106B0000E864FF1FFFFF0000E564FF1FE464FF1F50
:106B1000F7B50400808801F0D3FF0025A84203D018
:106B20000578A08802F008F81C4E3378002B1FD09F
:106B3000AB421DD11A4B28001978FFF777FF0028C8
:106B400018D000233370A3790820A778A688019372
:106B500005F002F9011E0DD0D0230370CA3B8370EB
:106B6000019B477086808371280005F0DDF801E005
:106B7000002DE8D1A0880B4B8200D358002B01D008
:106B8000FFF762FF1721A088FFF768FDA08801F0DA
:106B900027FDA08801F0FEFDF7BDC046E564FF1F9C
:106BA000E464FF1FEC64FF1FF0B587B01D000CAB61
:106BB0001B88070001930DAB1B88142002930EABBA
:106BC0001B88160003930FAB1B880091049310AB36
:106BD0001B88059305F0C0F8041E1AD0D02303705B
:106BE000CB3B47708370C670062229000430002D0D
:106BF00011D004F0A9FF019B21006381029B009842
:106C0000A381039BE381049B2382059BA37405F06E
:106C10008BF807B0F0BD04F0AFFFECE7F7B50093D9
:106C200008AB1B8807000C200D001600019305F02F
:106C300093F8041E13D0280001F042FF00280FD063
:106C40000078D0232370C93BA370009B21002381CF
:106C5000019B6770A580E680638105F065F8F7BD4C
:106C6000014B1878EDE7C0467043FF1F13B50400D1
:106C700064890389C2888188C0780094FFF7CEFFB9
:106C800013BD000010B5044C2068002803D004F0A8
:106C900063FD0023236010BDF064FF1FA122F0B547
:106CA000818892004A43384B384F1B6804009B1878
:106CB0009D2292009B18827989B01A603B68002B54
:106CC0005FD01D78324B1B68002B04D05B68002B13
:106CD00001D000209847260008363100E079FFF700
:106CE000B7FD237DE0710200E0780493638A2900F8
:106CF0000393238A0293E3890193A38800933300CB
:106D0000FFF752FFE378002B0BD1E289A379A1882A
:106D100002920196E27928000092012201F0DAFE47
:106D2000E0703B68002B20D0FFF7ACFF194D2878AE
:106D300000281AD0184B1978FFF778FE002814D0D5
:106D40002B78E67808200793A78805F005F8011E40
:106D500009D0D0230370CA3B467083708780867148
:106D6000079804F0E1FF00232B701721A088FFF79C
:106D700075FCA08801F034FCA08801F00BFD09B07F
:106D8000F0BD064B9DE7C0463409FF1FF064FF1FAE
:106D90000465FF1FE564FF1FE464FF1F7043FF1FCE
:106DA000F8B5070008000E0001F08AFE041E18D096
:106DB0002620FFF78DFC051E00D12578062004F063
:106DC000CBFF041E0DD00021062204F0D5FED023F7
:106DD0002370C23B21006770A370A680E8B204F064
:106DE000A3FFF8BDF0B585B001930AAB1B7807008F
:106DF00002930BAB1B7808000D000092039301F087
:106E00005FFE061E22D0102004F0A6FF041E1DD037
:106E10001022002104F0B0FE2620FFF759FC0028C4
:106E200000D13078D0232370C13BA370009B210098
:106E30002372019B67706372029BA580A372039B00
:106E4000C0B2E3720C9BE36004F06EFF05B0F0BDCE
:106E5000F7B50D00019001F033FE071E20D00E2083
:106E600004F07AFF041E1BD02620FFF731FC061E1B
:106E700000D13E78D0232380C53B0622A370F91DA4
:106E8000E01C04F061FE019B2A0063810123DD40C8
:106E90001A401D40210022736573F0B204F044FFD4
:106EA000F7BD0000F0B585B0029010000D0017008E
:106EB0000A9E039301F004FE041E31D0029B002BB6
:106EC0002ED1039B02795B0724D51223134304229E
:106ED000002E08D10B99002905D10C99002902D167
:106EE0000D9900291AD01A430D9B2271002B00D056
:106EF000C9E0002E00D1CFE0002D00D0CCE0606AC8
:106F0000002801D004F028FC1C21300004F094FE7D
:106F1000606205E002239A430E33D7E7934323715F
:106F2000654BBA00D458002C00D1AAE0002E10D036
:106F3000236A002B03D11C2004F086FE20625E4BE6
:106F4000BA00D358186A002803D01C22310004F07C
:106F5000FBFD0C9B002B12D0574CBB001D596B6ADC
:106F6000002B03D1162004F06FFE6862BB00E358CB
:106F7000586A002803D016220C9904F0E5FD0D9BF9
:106F8000002B11D04C4DBC006659B36A002B03D1C5
:106F9000142004F059FEB0622B59986A002803D0DF
:106FA00014220D9904F0D0FD380001F089FD051E72
:106FB00067D0414BBA00D358002B62D01A6A3420F4
:106FC000002A00D11C389A6A002A01D0143080B2FD
:106FD0000B9A002A01D01C3080B25B6A002B01D0D2
:106FE000163080B204F0B8FE041E4AD018220021E8
:106FF00004F0C2FD2620FFF76BFB0190002801D1B1
:107000002B780193D0232370029B200063700A2306
:10701000294EA370039BBD00A371AB59A780196AC9
:107020001830002905D01C22A06004F08DFD20003E
:1070300034307359996A002907D00300142214339D
:10704000E060029304F080FD02980B9B002B08D0B7
:1070500003001C221C330B992061029304F074FD81
:1070600002987359596A002903D01622606104F00E
:107070006BFD6B462100187904F056FE3800FFF7CF
:10708000E3FC05B0F0BD10220D9B0D991B69A01803
:10709000236204F059FD2CE70B9B002B00D13FE746
:1070A000012D00D03CE7606A002801D004F054FBB9
:1070B0001C210B982AE7C046EC64FF1F10B5044C56
:1070C0002068002803D004F047FB0023236010BD94
:1070D000E064FF1F0B4B07B51A68002A01D100209E
:1070E0000EBD6946531C012012780731FFF772FC70
:1070F0000028F4D002780123100018401A42EED084
:10710000EEE7C046FC64FF1FF0B51F4F01203B684F
:1071100087B0002B25D09B78059300F0B3FB0028A7
:1071200021D00A20FFF7D4FA04000B20FFF7D0FA91
:10713000164B05001E78731E9E413B68F6B2191D62
:10714000D878FFF757FB3B682900DA7A04330392BB
:107150009A7901930292009033002000059A04F07E
:10716000A3FC07B0F0BDFFF7B5FF002805D006204F
:10717000FFF7AEFA04000720D8E70820FFF7A8FAC7
:1071800004000920D2E7C046E064FF1FDC64FF1F53
:1071900070B50A4E040033780D00FF2B0DD004208B
:1071A00004F0DAFD011E08D0D0230370CE3B4570F9
:1071B0008370C470307804F0B7FD70BD8043FF1F4A
:1071C00070B5040006200D0004F0C6FD011E0AD0B3
:1071D000D0230370CD3B8370054B44701B688580C2
:1071E000187804F0A1FD002C01D0FFF767FF70BDF7
:1071F000E064FF1FF8B5264F06003B680D00112420
:10720000002B05D10522234B1B78134202D11224F7
:107210002000F8BD204A10241268002AF8D0127805
:10722000002AF5D0DB0719D52B789A1E012A1AD827
:107230000C2004F009FD132438600028E8D0002356
:107240000A22437029000670023004F07DFCFFF72B
:107250005BFF041E0AD0FFF731FFD9E700F012FBF5
:107260000028E1D1E4E7002BE2D0D0E70B4B1B78FC
:10727000032BCDD11D20FFF72BFA094B18800028D6
:10728000C6D0084B04211878074A04F07DFCBFE7FC
:10729000E064FF1FDD64FF1FFC64FF1FDC64FF1F51
:1072A000DA64FF1F0865FF1F60EA0000F7B501936D
:1072B000194B14001A78052306000F0012201A42F9
:1072C00021D0012920D1154B1D68002D1BD0022093
:1072D0001F2C18D8002C02D0019B002B13D0104B70
:1072E0001F221E706E1C0021300004F045FC019925
:1072F0002200300004F028FC310020002C70002F08
:1073000006D004F011FCFEBD064B12201D68DCE720
:1073100004F062FCF7E7C046DD64FF1FFC64FF1F5A
:107320008043FF1FF864FF1FF8B50F4E1224336827
:10733000002B17D01B780F3C834213D100250B4F35
:107340000221387804F0C8FB094B042138781D80ED
:1073500004F0C2FB074B28001D8033685C7004F00A
:107360006BFB04002000F8BDE064FF1F0865FF1FF1
:10737000F464FF1FDA64FF1F70B5012823D11B4C92
:107380002388002B03D01A4A1578002D07D0194BFB
:107390001B68002B02D01878FFF7C6FF70BD3B2B8F
:1073A00002D93C3B2380F9E7134E0221307804F0E8
:1073B00093FBFA222388920002215A43307804F08A
:1073C0000BFB2580EAE70B4B1B68002BE6D00B4B31
:1073D0001B785B07E2D5084B0221187804F07CFB90
:1073E0000022024B1A80FFF769FED7E7F464FF1F03
:1073F000D864FF1FE064FF1F0865FF1FDD64FF1FE7
:10740000F8B51E4D2868002803D004F0A5F9002324
:107410002B601B4E3068002803D004F09DF9002338
:107420003360184F05243B7818002040234221D0B8
:10743000154800F02BFA3B78234213D0202004F0AB
:1074400003FC2860002813D02022002104F094FBC4
:10745000202004F0F9FB041E306005D0202200211A
:1074600004F08AFB002004E0286804F075F92C6021
:107470001320F8BD00F00AFAF4E7C046FC64FF1FD1
:10748000F864FF1FDD64FF1F7443FF1F10B50A4C33
:1074900023681A1E0ED0002808D10130587004F05D
:1074A000CBFA002805D02368002B02D00021FFF77B
:1074B00087FE0122100010BDE064FF1FF7B5274EC4
:1074C000050033680191181E21D05C78244F012CEF
:1074D00030D1FFF7FFFD002825D02000FFF7F8F896
:1074E0000400412814D91F4B022118781E4A04F0C9
:1074F0004BFB1E4B3C3C1C80022233685A703B788D
:10750000002B14D128000199FFF75AFE0120FEBD7F
:10751000FA2292004243002AEED0124B0221187840
:1075200004F05AFAE8E7FFF7D3F80200F3E7002384
:107530003B70EBE73B78002BE8D1032004F00CFC18
:10754000011E08D0D0230370CC3B45708370336894
:10755000187804F0E9FBFFF7B1FDD7E7E064FF1FFF
:10756000D864FF1F0865FF1F60EA0000F464FF1F76
:1075700010B51749838802008B4220D011D81549D5
:107580008B4217D0144900205B1899B2012907D803
:10759000926811785A425341D8B2FFF7F9FD0120A1
:1075A00010BD0E4A00209B1807229BB29A42404110
:1075B000C0B2F5E783681878FFF768FFF0E78368E3
:1075C00099785A78090218781143FFF777FFE7E7AF
:1075D0000A20000006200000F8DFFFFFAFDFFFFFFA
:1075E000014B18707047C0468143FF1F10B5064C11
:1075F000207001F041FA207804F026F90521207866
:1076000000F062FD10BDC0460865FF1F0BB273B5E8
:107610000D00002B00DBC4E0884B187804F0ACFBB5
:10762000041E0ED00378912B0FD0A22B00D1A1E025
:10763000834B1878FF2852D0210004F075FB0028F6
:107640004DD180200002684076BD43780F2B76D064
:1076500013D8052B70D00E2BEAD18088794B984235
:107660002BD8794B98421BD8784B9842E0D1A3682D
:107670001878591CFFF774F838E03E2BD8D183787E
:10768000032B74D06CD8012B6ED0022BD0D1704B51
:107690001B68002B23D05B68002B20D098471EE08E
:1076A0006C4BC0180C28C3D804F0A6F81DC2C21534
:1076B0000BC20B0B0B3223C23C00674BC0180728D0
:1076C000B6D8664B1B68002B09D01B68002B06D070
:1076D000200098470AE0A3681878FFF7C7F8200051
:1076E00004F092F8ADE7A068FFF762F800289FD099
:1076F000F5E7A3681B78002BF1D0554B1B68002BD6
:10770000EDD01B68002BEAD0210055489847EDE7E3
:107710004F4B1B68002BE2D01B68002BDFD02100F1
:107720005048F3E7504B1B68002BD8D05B68002B08
:10773000D5D021004348E9E7FFF7EAF9CFE7808891
:107740004A4B984203D04A4B984200D070E7464BD0
:107750001B68002BC3D05B68002BC0D02100D5E78D
:10776000153B012BBBD963E7FFF798FAB7E7FFF7A3
:107770007DFAB4E73F4B1B78042B07D100236A4600
:1077800013800179408800F0C5FCA8E7364B1B68E0
:10779000002BA4D05B68002BA1D00100364898478D
:1077A0009DE7012421420AD0294B1B68002B04D0FD
:1077B0005B68002B01D000209847012043E78B072E
:1077C0000AD5264B1B68002B04D05B68002B01D028
:1077D00020009847022036E70421280008400D4287
:1077E00000D131E7254E3388002B21D0013B9BB2DD
:1077F0003380002B1AD1FFF7DBF800280AD0204B8A
:107800001C70164B1B68002B04D05B68002B01D04A
:1078100020009847FFF7C6F8694601F001FD684669
:10782000FEF7FEFF1D20FEF753FF308004200AE71D
:10783000024B187804F050F9F8E7C0460865FF1FBE
:107840008143FF1F0E2000000120000009100000EE
:107850000065FF1FFEDFFFFFAFDFFFFF0465FF1FB7
:107860000C2000000B200000E864FF1F0D2000002A
:1078700013200000DD64FF1FFFFF0000DA64FF1F1C
:10788000D864FF1F10B501F09BF910BD014B1860C3
:107890007047C0460465FF1F0B880020162B01D8D7
:1078A00017230420014A13807047C046B264FF1FAB
:1078B00000207047074A03001188814207D0918851
:1078C0000020994202D1013080001018704700203A
:1078D000FAE7C0461065FF1FF0B58F7806000D006F
:1078E000C5B01E2F15D1FFF7E5FF051E03D10024FB
:1078F000200045B0F0BD00223B003100C07800926E
:1079000000F0B2FB0400A81C00F0D2FBFF23EB70D8
:10791000EEE7264B062403931B78FF2BE8D0182FA5
:10792000E6D87B08224A013BDB0002929A58944633
:10793000002ADDD0029AD3185B68002BD8D00878D3
:10794000002802D14B78012B02D10624122FCFD16F
:1079500007AFAB88697800976446AA68A047041E01
:10796000C6D1AB78029A5B08013BDB00D318390023
:1079700030005B689847041E0BD1AB78042BB6D05F
:10798000039A310010782200009700F06DFB04008C
:10799000AEE76A78002AABD1AA7805A93B880871BE
:1079A00030000A704B80FEF747FBA0E78443FF1FBF
:1079B0006CBF00111D4B37B5050098420BD0002954
:1079C0000AD1FFF777FF002805D11948FFF772FFAA
:1079D000002800D0058037BD01291AD1FFF76AFFC2
:1079E000041EF8D001235B420380A378FF2BF2D062
:1079F000FE2B07D00023E0781422009329001E33C9
:107A000000F032FBA01C00F053FB01235B426380BB
:107A1000E1E70229DFD1013901F0BEF80028DAD10F
:107A20002800FFF747FF041EDFD1D4E7FEFF000068
:107A3000FFFF0000022210B5074B52421A80074890
:107A400001325A809A80DA8000F07EFA044801F010
:107A500025F8002010BDC0461065FF1FD978001121
:107A6000B57900110388F7B50400002B02D1022577
:107A70002800FEBD42680221137825485268FEF7AF
:107A8000A5FD00282ED0234F01253A88002AEFD0EB
:107A9000802321885B0201259B1A9942E8DC0C2097
:107AA00004F0D2F8061E31D03B8822889C46002381
:107AB0001800019561469DB2491989B2AA421BD8A6
:107AC000002801D062443A8000233000082208C018
:107AD000210004F039F8104A1368002B13D1002557
:107AE0001660C5E76268022113780C485268FEF7F9
:107AF0006DFD0028C7D1BAE760681D0140194181BA
:107B000001330198D6E71A001B68E6E71325AFE7B3
:107B1000DABF00118243FF1F0C65FF1FD8BF0011A1
:107B2000014B18707047C0468443FF1F14230A009E
:107B300010B51A40194204D00122102101F048F872
:107B400010BD4B06F9D4012088434000F8E710B57A
:107B500014008B0604D50122102101F039F810BD64
:107B600008230A001A40194202D14BB2002B0FDA47
:107B7000102101F02DF8002808D02300F2331B78E3
:107B8000002BECD0F1342378012BE8D10020E6E77C
:107B900003208907FAD4E2E7F0B51F00184B85B03F
:107BA0001C68019002910392002C27D1200005B09F
:107BB000F0BDA5683301ED186B89019A934211D38A
:107BC000029A93420ED8002F04D10A9B002B10D1A9
:107BD0002C00EBE73B002978039A6868FEF7F6FC77
:107BE0000028F2D10136B6B2A388B342E1D82468A6
:107BF000DAE7A3680A9A5B891380E9E70026F3E7CE
:107C00000C65FF1F37B50C000A8849880123914293
:107C100017D3002A15D0651D23792A0002210A48AE
:107C2000FEF7D4FC102300280BD02379618820882C
:107C300000242A000094FFF7AFFF0A23A04200D0DF
:107C4000230018003EBDC046DABF001113B50A007C
:107C500008884988012388420BD8002809D00024CD
:107C6000137905320094FFF797FF0A23A04200D052
:107C70002300180016BD13B50A000888498801239F
:107C800088420BD8002809D00024137905320094CB
:107C9000FFF782FF0A23A04200D02300180016BD80
:107CA000F0B58BB003904A8808880E000123824209
:107CB00055D3002853D00023012704AC23700022A1
:107CC000718813000092FFF767FF051E3ED02078F1
:107CD000002835D12B78022B18D167706A89830070
:107CE0000130E31880005A8069680222201803F0EE
:107CF0002BFF23780133DBB22370042B19D93B000F
:107D00006889013080B2002BD9D01FE00223637054
:107D1000122358436A89231804305A806968102254
:107D2000201803F011FF23780133DBB22370002BFE
:107D3000E5D10C4A6B899B185A425341DBB2DFE70D
:107D40006378012BE4D12B78022BC7D022780A2349
:107D5000002A04D021000398FEF798F900231800A8
:107D60000BB0F0BD0100FFFF0F4BF0B50400186829
:107D7000002816D083685D89A54207D88288AE188E
:107D8000B44203DA12019A18934201D10068EFE776
:107D90001E005F891036A74204D1002900D00D8053
:107DA0001800F0BD3300EFE70C65FF1F70B505004C
:107DB0000C0008880021FFF7D7FF03000120002BEB
:107DC00004D022002800197AFFF7C1FE70BDF7B574
:107DD0000C00002501902300EE331B78AB4201D844
:107DE00000200AE06B00E65A00213000E718FFF798
:107DF000BBFF002802D126800130FEBD017A019828
:107E0000FFF794FE002802D03B882380F5E7013578
:107E1000EDB2E0E710B5040008880021FFF7A4FFE9
:107E200003000120002B03D02000197AFFF77EFE0B
:107E300010BD0000054B1B68002B01D1180004E0A9
:107E40009A6852898242F6D1988870470C65FF1F64
:107E5000F0B50E27002687B0039302ABFF183E80D3
:107E600005001F4B40891400984207D02B78013041
:107E700000976A6880B2FFF78FFE060002212B7818
:107E800018486A68FEF7A2FB00280FD06C89200012
:107E9000FFF7D0FF002802D0013C0419A4B2039BD5
:107EA000002B00D01C80300007B0F0BD02212B78E1
:107EB0000D486A68FEF78AFB0028E7D102212B787B
:107EC0000A486A68FEF782FB002807D0002EDED041
:107ED0003B88A342DBD17489013CDFE76C89DEE794
:107EE000FFFF0000DABF0011D8BF0011D6BF00119C
:107EF00010B50C00FFF7DEFC03000220002B0AD0B7
:107F0000002C00D023609B781720FE2B03D0013873
:107F1000FF2B00D1002010BD73B50D0001A9040096
:107F20001600FFF7E5FF172805D0002E04D1290021
:107F30002000FEF727F976BD01221021200000F075
:107F400047FE0028F3D0F6E7014B18607047C046A3
:107F50001C65FF1F37B56B469D1D01000400022202
:107F6000280003F0D1FC2B88B02B0ED12379122BE3
:107F700009D12300FA331B78012B06D10121608837
:107F800000F0E0F801E01B2BF8D037BD10B5054B31
:107F90000421187000F098F8FFF74CFDFEF770FB15
:107FA00010BDC0462065FF1F0020F0B50BB20F00CA
:107FB00087B0834234DA274B187803F0DDFE051EC4
:107FC0002BD00378A02B25D103AE3100FEF7E4F8C7
:107FD000041E0BD1B378DB0724D51F4B06341B6876
:107FE000002B03D03100688898470400A868002857
:107FF00001D003F0F9FC002C08D1184A039B134070
:10800000174A934206D0B3781B2B03D0012168880E
:1080100000F098F8280003F0F7FB80200002784079
:1080200007B0F0BD0F4B1B68002B10D031006888E3
:108030009847041EDAD07378002BD7D1B27801A903
:108040000A704B800C716888FDF7F6FFCEE70624B6
:10805000F1E7C0462065FF1F1865FF1F00FFFF0006
:10806000000112001C65FF1FF7B50190FC200D00F8
:1080700017001E0003F070FE04001320002C12D025
:10808000B02320002370089BF4226770658026715E
:108090000830002B08D0190003F056FD210001988C
:1080A00003F042FE0020FEBD089903F065FDF5E7F0
:1080B00010B5041E06D00078FD2803D803F054FB49
:1080C000FF23237010BD00000A1F93B210B50400F7
:1080D0000220032B05D882400020024BD1529B186E
:1080E0009C7010BD4065FF1F0B8870B5043B0400F9
:1080F0000D000220032B0BD80121200000F04CFDC5
:1081000003001420002B03D02900200000F0DEFB28
:1081100070BD000007B51300034A00920A00012158
:1081200000F02CFC0EBDC0465183001107B5019232
:1081300003220092024B0A00122100F049FC0EBDFE
:10814000CF83001107B56B4601AA11800449D8807E
:1081500008780633012802D1190003F0CDFC07BDD1
:108160002165FF1F0C4B10B518700023FF210B4A2F
:108170001380138193819380094A53801370517245
:1081800093819372D174D3821375517703F01CFDE0
:1081900000F0FCF910BDC0465065FF1F4065FF1F91
:1081A0002265FF1FF0B58DB06B46002003910C22B5
:1081B0009B5E834200DBB0E05D4B187803F0DCFD92
:1081C000051E00D1A4E00378902B00D09DE006AFFF
:1081D00001004688380000F013FA7968040000298D
:1081E00000D19CE03B88052B6ED13B89032B1CD929
:1081F00005AC200000F0A2F86288172A61D83989FE
:10820000131D994231D17968237804310291D9073D
:1082100038D5607800F08EF9071E06D00023037170
:108220002378012B08D0132B23D0A868002800D175
:1082300078E003F0D9FB75E06288029909A800F0A4
:10824000A6F80290380000F08BF909AA2378387A52
:108250000192002231000092029A00F012F93800D7
:1082600000F064F9029B002BDFD0300000F080F9B1
:10827000DBE70378032BD8D16288029909A800F0C4
:10828000D6F8DEE7122B13D1029909A800F0B5F851
:10829000021EEAD127498B88002BC6D0887909A90C
:1082A0002378019161780091310000F0EAF8BCE791
:1082B000002302AA93833000617809AAFFF72AFFFE
:1082C000B3E71D4B0993F6E7042B02D09A1F012A4E
:1082D000ABD8184A043B9B00995A0029A5D0D21864
:1082E000907831003A0000F0AEF800289DD13B882C
:1082F000042B03D001213000FFF724FF012C04D10F
:10830000A868002801D003F06FFB280003F07CFA76
:108310008020039B0002434018000DB0F0BD0128EF
:1083200000D182E701213000FFF70CFFEDE7C046E6
:108330005065FF1F4065FF1F010017000B78037099
:108340004B784370CB788A781B0213434380704785
:108350000A88030002700A88120A42700A88012AF9
:1083600006D14A8882704A88120AC2700420704777
:1083700002208242FBD14A8804309A704A88120A4D
:10838000DA708A881A718A88120A5A71EFE710B572
:108390000400012082420CD94B780A781B02134357
:1083A0002380834206D1CB788A781B0213436380F3
:1083B000002010BD022BFBD1CB788A781B0213431F
:1083C00063804B790A791B021343A380F0E70B8883
:1083D00003700B881B0A43704B8883704B881B0A01
:1083E000C3708B8803718B881B0A4371CB888371A0
:1083F000CB881B0AC3710820704703000120082A9C
:1084000014D14A780878120202431A80CA78887810
:10841000120202435A804A790879120202439A8072
:10842000CA798879120202430020DA80704710B5B9
:1084300004000120022A05D100204B780A781B0293
:108440001343238010BDF8B5060010200F0015005F
:1084500003F082FC04000120002C0ED0A0230C228B
:10846000290023806780201D002D07D003F06CFBBE
:108470002100300003F058FC0020F8BD03F07CFB25
:10848000F6E7F7B51E00009008AB142017001D7822
:10849000019103F061FC041E12D0A2230370019B22
:1084A00047704380099B057146710C220830002BF0
:1084B00007D0190003F048FB2100009803F034FCBA
:1084C000F7BD099903F058FBF6E737B5041E0FD046
:1084D0004388002B0CD00025C1881323007A172273
:1084E00001950095FFF7CDFFFF236580637225702E
:1084F00037BD000010B50C4904004A88002A09D095
:108500008B89002B05D00020CB8A0222834201D028
:1085100010BD012213000A20434300204032C854FA
:10852000C81842800472F3E72265FF1F00234380CE
:1085300003707047094B00211A0010B55C88002CAD
:1085400006D01C79844203D10A234B43D01810BDB6
:1085500001310A330329F1D10020F8E72265FF1F1A
:1085600010B50400407A03F0FFF8FF23637210BDDA
:108570007047043010B580B203F076F9002803D0BC
:108580000421494203F028F910BD000070B5002510
:10859000104CA0682580A581A580A84202D003F0D8
:1085A00023FAA56000250C4C0C4B606D1D80230048
:1085B00058331D70A84202D003F016FA65650025F5
:1085C0006068002801D003F00FFA013508340A2D45
:1085D000F6D170BDE865FF1F8C65FF1FDC65FF1FCE
:1085E00070B5041E09D1054D2880A881A880A8680F
:1085F000002802D003F0F8F9AC6070BDE865FF1FF9
:10860000F0B54B8885B00193002343600A790500DB
:108610000F00022A00D07BE0CA88032A17D98B6892
:108620005E7819783602DC78D8790E4399781B7A0F
:1086300024021B020C43034353495BBA0B80331DD6
:1086400093421ED1042C04D0631F022B0ED90120AB
:1086500015E0019A4D4B1201D35A002B06D0019818
:10866000FFF7BEFF4A4A1369013313610421B8685A
:108670002E812C80494203F0AFF86860002005B0DD
:10868000F0BD434D042C06D0631F022B0FD9EB68BD
:108690000133EB60DBE7019A3C4B1201D35A002B0C
:1086A00005D00198FFF79CFF2B6901332B61374BF5
:1086B00030000293019B029A1B0101930023019950
:1086C0008C468B52130063449C8003939E81FFF77A
:1086D00050FF039B041E986016D00421B8684942DD
:1086E00003F07AF8FA880100043A200003F02CFA2B
:1086F0000199029AFB888A5A043B9B18029A8B5272
:108700002B6801332B60A2E7AB690133AB619EE7B5
:108710001E4B0293019B1E01029BF35A002B2DD08E
:1087200002998C19A068002828D0012A26D1FA883D
:108730009B189BB27352A189994217D39B1AC018F8
:10874000B96803F001FA029BA289F35A934200D060
:108750007DE700222B81A3882B80A3686B60029B9E
:10876000F2520B4A53680133536070E7084A93682A
:10877000013393600198FFF733FF68E7044A5369B8
:1087800001335361F6E7C0465265FF1FE865FF1FDE
:108790005865FF1F70B5051E15D10B4C0B4B18808B
:1087A000230058331870606D002802D003F01CF9C4
:1087B0006565250050356068002801D003F014F984
:1087C0000834AC42F7D170BD8C65FF1FDC65FF1F1C
:1087D000F0B51700A12285B0920001934243394BB6
:1087E00006001B680C009B18D933FF331D78FDF77A
:1087F00041FF0430854204DD3000FDF73BFF0430CB
:10880000C5B2BD4207D33A0000213000019B03F0FE
:1088100053F805B0F0BD2900380003F075FA2300C5
:10882000C6B250331E700393019B29006365380064
:1088300003F032F9CBB20293002B02D0039B013636
:108840001E7000262300503303931B78B34204D8D4
:10885000606D002831D10020DBE7029A2800002A51
:1088600004D0013B1000B34200D02800F700E71904
:10887000387003F091F9786000280ED03A780199A9
:1088800003F062F9019A3B780136D3180E4A01933E
:10889000D369F6B20133D361D4E7039B18706065E6
:1088A000A74205D1084A1320D36A0133D362B0E747
:1088B000606803F099F80834F2E703F095F80023B4
:1088C0006365C8E73409FF1F5865FF1FF7B50D0042
:1088D00007000421686802F07FFF2B890400037001
:1088E0002B891B0A43702B8883702B881B0AC3704B
:1088F0002E8902250436F6B2F42E15D81B4B9F4262
:1089000014D10C2003F028FA1135011E0CD090234D
:1089100003708E3B0371043B4380154B8460C6801B
:10892000187803F001FA00252800FEBD5C237B4384
:10893000104AD3180093583301931B78002B0FD1A2
:108940000300320038000099FFF742FF019B050049
:108950001B78002BE8D13800009902F0B5FFE3E75F
:10896000054A0725536A01335362DDE7FEFF000025
:108970005065FF1F8C65FF1F5865FF1FF0B587B05E
:10898000009017200F0016000193FFF7F2FD13254A
:10899000041E19D00C98031E02D00199201D98477F
:1089A000030AE370052302AAA070043090812770A7
:1089B0000098667003A993800494FFF787FF051E53
:1089C00002D0200003F010F8280007B0F0BD00002E
:1089D000F0B587B01F000CAB1B7803910593012104
:1089E0000DAB06001C78049200F0D6F81425002880
:1089F00021D02000FFF77EFD0135041E1BD0114958
:108A0000059B0A7803700132D2B2131EC68001D1D1
:108A100001231A000B7022713000049B0399009708
:108A2000FFF7ACFF051E09D1230021000648074AC5
:108A3000093302F039FF280007B0F0BD002363803E
:108A40002370F8E75465FF1FCB84001130750000D8
:108A5000F8B505000E00064C064F2368002B02D027
:108A60003100280098470434BC42F6D1F8BDC04616
:108A7000F865FF1F0C66FF1F0123064A5B42538007
:108A8000002313715362044A136053609360D360F0
:108A9000136170470C66FF1FF865FF1F020000237B
:108AA00010B506499C000859002801D1625010BD3C
:108AB0000133052BF6D11320F9E7C046F865FF1FF7
:108AC000034A5388181A43425841404210407047A5
:108AD0000C66FF1FF0B585B002930AAB1F780CAB94
:108AE0001B88009008000E0001920393FFF7E8FF37
:108AF00005001120002D1BD10E48FFF7E1FF0400F7
:108B00001520002C14D006220B99A771E01D03F04C
:108B10001BF8019B30002371029B29006371009BAD
:108B200066802370039B6562E381FFF791FF280055
:108B300005B0F0BDFFFF000010B5FFF7C1FF040056
:108B40000220002C12D060880121FFF781FF606AAB
:108B5000002801D002F000FE28220021200003F0AE
:108B60000BF8012300205B426380207110BD0000E0
:108B700030B5074A074C5588010013780020A542FC
:108B800004D05B1A59424B415842104030BDC04698
:108B90000C66FF1FFFFF0000084A10B501230C0000
:108BA000904208D0FFF78CFF031E04D003792340C6
:108BB0005A1E9341DBB2180010BDC046FEFF0000F4
:108BC000024B1879431E9841C0B270470C66FF1FD4
:108BD00070B504000D001600FFF772FF002804D1E5
:108BE0000D4B9C4200D0143070BD416A03790520C2
:108BF000002907D012221A40102A02D10520002E87
:108C0000F2D10F20DB06EFD5897E0C20A9428941E5
:108C1000494249420840E7E7FEFF0000030010B563
:108C2000002800D110BD0348034A41889142F9D081
:108C30009847F7E70C66FF1FFFFF0000002330B5E1
:108C4000C45CCD5C6C40D4540133102BF8D130BDE2
:108C50000F23002210B5C45C64002243CA54C25CD6
:108C6000D209013BF7D210BD0200010010B520323D
:108C7000103102F081FD10BDF0B58BB003901020D3
:108C800005931700049102F0DFFF0090102002F01E
:108C9000DBFF009B13240190002B05D000280CD192
:108CA0001324009802F058FD019B002B02D01800FD
:108CB00002F052FD20000BB0F0BD102002F0C4FF06
:108CC0000600102002F0C0FF13240500002E00D182
:108CD000AEE0002819D01022002102F04DFF320032
:108CE0002900039802F048FD041E0ED133787F2B33
:108CF00051D830000099FFF7ABFF009B1B787F2B0A
:108D000053D801990098FFF7A3FF300002F024FD2B
:108D1000002D02D0280002F01FFD002CC1D1102030
:108D200002F092FF0600102002F08EFF0290002E4B
:108D30007CD0002878D03A000F3223000125121190
:108D400005D00F333B4015B25A4253411BB26A1E45
:108D50001201002B33D0049BD2B298180099029ACA
:108D6000FFF76CFF013D10220021300002F004FFEC
:108D7000ADB2049F2D017D19AF4242D0002C33D0FB
:108D8000300002F0E9FC029B002B00D189E71800BB
:108D900002F0E2FC85E729003000FFF759FF2800C8
:108DA0002549009AFFF74AFFA7E729000098FFF737
:108DB0004FFF28002049019AFFF740FFA5E70F2148
:108DC0000F4004998A18D9B28F4208D9D15C06A8FD
:108DD00019540133102BF6D1029A0199C0E7791A80
:108DE00048424141C901F2E73900300006AAFFF7C5
:108DF00025FF3200039806A902F0BEFC10370400DC
:108E0000BAE7002CBCD13000029906AAFFF716FF82
:108E1000320006A9039802F0AFFC082204003100DA
:108E2000059802F091FEABE71324A9E71324AAE703
:108E3000002800D06EE733E7E0BF0011F0B58BB03B
:108E40000F0016000225009000283FD0002A3DD0D8
:108E50000B1DDBB21800029302F0F6FE1135041E62
:108E600034D0FDF747FD05003A000099201D02F0BF
:108E70006BFDEBB20393E3702B0CDBB22F0A009374
:108E80006370FFB22B0E2370A7700193FDF72CFDCA
:108E90001022010006A802F057FD2100029A04AB3F
:108EA00006A8FFF7E9FE051E0DD1039B08223370CB
:108EB000009B04A9B370019B7770F370301D02F022
:108EC00043FDFDF71DFD200002F046FC28000BB01D
:108ED000F0BDF0B58FB00D00149E03900492059381
:108EE000002A03D1022420000FB0F0BD002EF9D0DB
:108EF0000398FFF7E5FD1424071EF4D07278337849
:108F000012021A43B3781B041343F27812061A4371
:108F1000036A0192934201D30133E3D1002D03D0C0
:108F20003B7901249B07DED50822002106A802F028
:108F300023FE059B13240433DBB21800029302F0D6
:108F400083FE051ECFD0059A0499043002F0FCFC84
:108F500004223100280002F0F7FC39001022103101
:108F60000AA802F0F1FC2900029A06AB0AA8FFF752
:108F700083FE041E0FD1082206A908A802F0E4FC13
:108F80000822311D08A802F097FE012807D1019997
:108F90000398FDF7C9FC280002F0DEFBA3E70124DB
:108FA000F9E7000070B51C4C05002368181E10D0AE
:108FB000002D14D11A78002A0CD1981C083202F026
:108FC000C3FD02F059FD0135002808D123681D704A
:108FD000012070BD0A331800082202F0B5FD236895
:108FE000002BF5D0122002F0B7FE061E0DD0C123D3
:108FF00021680370457002311022023002F0A4FD96
:1090000023683100587802F08FFE206802F0A4FB3C
:1090100000232360DCE7C0463466FF1FF8B5040078
:109020002020FDF755FB0D4EA700BB590500002B76
:109030000DD000280BD0D878FF2809D108492A0084
:109040000C55F35907480333611802F02DFCF8BDA5
:10905000290002F0D9FC0028F0D1F8E75066FF1F84
:109060003866FF1F75A2001170B5064D8400635964
:10907000002B05D0D87802F077FBFF226359DA7015
:1090800070BDC0465066FF1F70B506008CB00C0066
:10909000150000213022684602F06EFD31001022DA
:1090A000684602F051FC1D2021000322684402F0B2
:1090B0004BFC6846FFF7D8FD2D2104000322280051
:1090C000694402F041FC20000CB070BDF0B507000F
:1090D000160097B001931CAB1D7830221EAB009197
:1090E0000AA800211C7802F047FD102239000AA8C6
:1090F00002F02AFC1022002102A802F03DFD072206
:10910000310002A802F020FC072202AB9818631E6F
:109110009C41019902F018FC02AB9C732B005A1E73
:10912000934102AAD3730021102206A802F024FD65
:1091300006221D9907A802F007FC1A2002ABC018EE
:1091400006221F9902F000FC102200990EA802F0DE
:10915000FBFB102202AB0EA908781C78013A604094
:10916000D2B2087001330131002AF5D10AA8FFF705
:109170007BFD102212A904000EA802F0E5FC1022CB
:1091800006AB0EA908781D78013A6840D2B2087083
:1091900001330131002AF5D10AA8FFF765FD044328
:1091A00010222098E4B212A902F0CEFB200017B0E2
:1091B000F0BD70B50E0014008CB00100102268469E
:1091C0001D0002F0C1FB3100082204A802F0BCFB24
:1091D0002100082206A802F0B7FB6846FFF744FD0D
:1091E00004001022280008A902F0AEFB20000CB0F9
:1091F00070BDF8B506000D0000243719AC4200D34D
:10920000F8BD02F0E1FB030A3B70631CDBB20137DF
:109210009D4203D90234F054E4B2EEE71C00EDE7BE
:1092200073B506000C000225002819D0002917D0BC
:10923000032101A8FFF7DDFF6B469A793F231A400F
:10924000013313436A463000937101A92200FFF7EE
:109250001BFF051E04D10322E01C01A902F074FCCF
:10926000280076BD03785807DA08C00FD2008000C6
:109270009B0710439B0F1843C0B2704707230B4056
:10928000C908C9000B4303707047000070B50400A3
:10929000FFF7EAFE134DA4006359002B21D0186A92
:1092A000002801D002F058FA2B59986E002801D0FE
:1092B00002F052FA2B59D86E002801D002F04CFA75
:1092C0002B59186F002801D002F046FA2B59586F1D
:1092D000002801D002F040FA285902F03DFA00239C
:1092E0002B5170BD5066FF1F0E4B8000C35870B5E8
:1092F0000C00002B0FD09D68002D0CD02B78201D6A
:109300000B706B784B70A97CFFF7B8FF2B7E237234
:109310006B69E36070BD10220021200002F02CFC7C
:10932000F8E7C0465066FF1F014B18607047C04603
:109330004C66FF1F074A03008000825810B5002AC0
:1093400006D0D088984203D1012901D1FFF79EFFB2
:1093500010BDC0465066FF1FF0B5264E95B0870081
:109360000B93BB590500099112200A92002B31D0B2
:10937000D888FFF7A5FB04001420002C2AD0280071
:1093800010A9FFF7B1FFBB591E781D6A002E23D02C
:109390000895FDF7EFFA07000020FDF7F1FA0790B6
:1093A000A379E61D069310AD0CA9089800F0E2FA27
:1093B0000EA9280000F0D7FA0B9B0A990493069B8C
:1093C00009980293079B0396019300970EAB0CAA92
:1093D000FFF77CFE15B0F0BDFDF7CCFA069030002B
:1093E000FDF7CEFAE31DA779079310AB06000893AB
:1093F000DAE7C0465066FF1F30B50C4C85002A598D
:10940000030085B00120002A0ED018006946FFF73E
:109410006BFF2B591A78D888054B002A00D1054BD1
:109420006A46072100F0D9FB05B030BD5066FF1F2A
:10943000679900117599001130B5094C85002959BB
:1094400085B010226846253102F07EFB2A59112191
:10945000044BD0886A4600F0C0FB05B030BDC04662
:109460005066FF1F119A001130B5094C850029592B
:1094700085B010226846353102F066FB2A59112169
:10948000044BD0886A4600F0A8FB05B030BDC0464A
:109490005066FF1F4F9A0011F7B54D4F8600102000
:1094A000F4590D0002F0D0FBF3592062186A132220
:1094B00000286CD0033A29009C6802F045FBF35960
:1094C0001A780192002A58D11E6A227D317B944677
:1094D00051400122019F114201D167461740217D71
:1094E000914339432175377B4F40BC466046002786
:1094F000800701D44F081740012102208F40227DB0
:1095000082433A432275377B5740BC46604600276A
:10951000400701D497080F400420227DBF008243FA
:109520003A432275627D002794466046727B424032
:109530000A4201D167460F400121627D8A433A43C6
:109540006275777B5740BC4660460027800701D490
:1095500057080F400220627D7F00824317436775E2
:10956000767B00227E40760701D4BA080A400426A2
:10957000617D9200B1430A4362756A78002A08D07F
:109580006278002A05D005220533DA770022100020
:10959000FEBD04222979114205D1A17C114202D1DC
:1095A0000533033AF1E7019A21782C78002A02D199
:1095B0000A002100140018220429E8D8042CE6D857
:1095C00005206043034A05331218525CDDE7C046AC
:1095D0005066FF1FF0BF001110B50A001121024BA9
:1095E00000F0FBFA10BDC046AB9A00110B0030B57D
:1095F00087B001AD2B806B4604001100981D082236
:1096000002F0A2FA2A000B212000024B00F0E5FA3A
:1096100007B030BDD39A001110B50A001121024BDA
:1096200000F0DBFA10BDC046279B001113B50B00FC
:1096300011006A4613706B4604000622581C02F0A3
:1096400083FA6A4608212000014B00F0C6FA13BDD8
:10965000479B001110B50A001121024B00F0BDFA22
:1096600010BDC046979B00117FB505000B4BAA00AB
:10967000D4580800002C0FD0666F237FE288217831
:109680000396266F0296E66E0196A46E0094FDF78F
:1096900009FC2800FFF7FAFD7FBDC0465066FF1F9A
:1096A00010B51721FFF7E0FF10BD000070B50A00EC
:1096B0000D00064B0221040000F08FFA0600297805
:1096C0002000FFF7D1FF300070BDC046779A00112F
:1096D00070B586B000236A461370836804001D7855
:1096E000681E0A2859D801A902F00EFA0606333777
:1096F0003B3F43474B4F5300180000F042F906230D
:1097000012284BD000281BD16088FFF7D9F9082315
:10971000002813D04279002A47D1264B1A78072314
:1097200012070BD5244B1A680723002A06D01668A7
:10973000002E03D0290001AAB04703006A46137027
:109740006B461B786088002B2AD1FFF767FC06B0B8
:1097500070BD180000F06CF9D4E7180000F087F92C
:10976000D0E7180000F093F9CCE7180000F0ADF94D
:10977000C8E7180000F0C3F9C4E7180000F0F6F9D4
:10978000C0E7180000F0F6F9BCE7180000F013FA83
:10979000B8E7180000F013FAB4E707236A4613701D
:1097A00069466088FFF782FFD1E70523012AC5D10A
:1097B000024BB8E7DD64FF1F4866FF1F4C66FF1FC2
:1097C000F8B52C4F8600F35904000D00002B40D053
:1097D000DA8882423DD15A78062A33D11A78002A93
:1097E0002ED0012099681A6A097D014206D0157BA6
:1097F000054203D007225A700120F8BD0220014221
:1098000004D0157B054201D00922F4E7042001426F
:1098100004D0127B024201D00B22ECE7164B1B68EE
:10982000002BE9D05B68002BE6D020009847BB599D
:1098300000215B78122BDFD12000FFF715FFDBE75B
:109840000E4BECE7112A04D1002900D03225290063
:10985000F2E7002D08D12000FFF732F9002803D0ED
:10986000102302791343037121002800FDF798FAB1
:10987000C2E7C0465066FF1F4866FF1F4C66FF1FC9
:1098800070B50E4E8500AB590400002B13D01B7829
:10989000002B11D10A4B1B68002B04D05B68002BF6
:1098A00001D02000984773595B78122B03D1002117
:1098B0002000FFF7D9FE70BD024BECE75066FF1F9A
:1098C0004C66FF1F4866FF1F094B8000C3581020DD
:1098D000002B0CD01A6A002A09D09B68002B06D0F6
:1098E000127A1B7E101C9A4200D9181CC0B2704715
:1098F0005066FF1F70B503000D0014000220002AFF
:1099000030D000292ED013700B78081D53704B787F
:109910009370FFF7A7FCE070012002212B7A2371DE
:109920006B7B034063716A7B0A40134304226371BB
:109930006E7B1640334363716E7BF608F60033434B
:1099400063712B7B0340A371287B014000200B43F4
:10995000A371297B0A401343A3712A7BD208D2004A
:109960001343A37170BD10B50A0001000120FFF779
:10997000C1FF10BD10B50A0001000220FFF7BAFFB9
:1099800010BD70B506000C000220002E30D000295A
:109990002ED07378201D0B70B3784B70F178FFF7E1
:1099A0006DFC01223579257271794B100800134046
:1099B000934010400343881010408000C9080343BF
:1099C000C9000B436373B1794B10080013409340F7
:1099D00010400343881002409200C9081343C90095
:1099E0000B4321202373FCF773FE854201D2122022
:1099F00070BD2220257AFCF76BFE8542F7D82378CC
:109A00001820042BF4D86378012BF1D80020EFE75D
:109A1000030010B50220002909D0002B07D0032233
:109A2000481C0A7019000D3202F08EF8002010BD9B
:109A300003000222080010B5002B06D0002904D034
:109A40000E32591C02F080F80022100010BD0300F5
:109A500010B50220002909D0002B07D00422481C91
:109A60000A7019000C3202F06FF8002010BD10B51A
:109A7000FFF7DEFF10BD03000220002906D0002BF7
:109A800004D0052200200A701B784B707047030039
:109A90000220002B08D0002906D05B7800200B7034
:109AA000013B082B00D918307047030010B5022085
:109AB000002909D0002B07D00622481C0A70190083
:109AC0000A3202F041F8002010BD10B5FFF7B0FFD8
:109AD00010BD02000B00022010B500290ED0002A94
:109AE0000CD007211970118859701188090A9970D2
:109AF00011180822D81C02F027F8002010BD03001E
:109B00000A00022010B5002B0CD000290AD0997849
:109B10005878090201431180901CD91C082202F0D8
:109B200013F8002010BD030010B50220002909D051
:109B3000002B07D00822481C0A701900921802F066
:109B400003F8002010BD02000B00022010B5002910
:109B50000BD0002A09D009211970117818185970F2
:109B6000511C062201F0F0FF002010BD10B5FFF7D8
:109B70005FFF10BD02000B00022010B5002A09D0C3
:109B8000002907D05178197011180622581C01F0CD
:109B9000DBFF002010BD030010B50220002909D012
:109BA000002B07D00A22481C0A701900063201F067
:109BB000CBFF002010BD10B5FFF73AFF10BD02002B
:109BC0000B00022010B5002A06D0002904D018008E
:109BD0005178FFF753FB002010BDF0B585B017009A
:109BE0001E006A4606230500080091819380FEF757
:109BF000C0FC1324011E02900CD03800B047041E94
:109C000005D1280001A9FEF76FFA041E02D00298C0
:109C100001F0EAFE2800FFF701FA200005B0F0BDD0
:109C2000F0B504008BB0019115000021102202A8AC
:109C300001F0A2FF334EA700B85900283CD0C388DA
:109C4000A34239D10378002B36D14278062A18D1A5
:109C500002000100553235310C3006ABFFF7A9FA8E
:109C6000002829D12000FFF72FFE020006A902A834
:109C700001F06AFF200002A901F04EFE01200BB0A6
:109C8000F0BD816E002917D00B8A112A28D19D4280
:109C90000ED101981231093A02F00EF8012807D1CD
:109CA000BB5920009D6EFFF70FFE29000200DEE782
:109CB00032212000FFF7D8FC2000FEF701FF061E2E
:109CC0001BD0416A002918D00B8AAB4215D108225B
:109CD0000198123101F0F0FF01280ED1716A0AE0FB
:109CE0009D42E9D108220198123101F0E5FF0128D7
:109CF000E2D1BB59996E8A7EB9E7200001F074FF6A
:109D0000BCE7C0465066FF1FF0B56B4D87007E591B
:109D100085B0337802900393002B00D087E0B368BE
:109D2000346A01937078062817D101221B7D1342F3
:109D300002D0217B114218D10222134202D0217B92
:109D4000114251D10422134203D0237B134200D08D
:109D50008BE0019B5A7DEB5991E007380428F8D835
:109D600001F0D2FE032E42678300B36E002B03D1B5
:109D70001C2001F069FFB066EB599C6E002C1CD0D2
:109D800010220021200001F0F7FE0298FFF79CFD51
:109D900001002000FFF72DFA01F016FE20822000BE
:109DA00008211230FFF725FA0298FFF78DFDA07603
:109DB000EB592100D888FFF70FFC0822EB591CE073
:109DC000B36E002B05D01A00198AF0881232FFF703
:109DD0000DFC0222019B197DEB5911423DD0207BE5
:109DE00010423AD0073208E0F488FCF7DBFD0100AE
:109DF0002000FFF711FC0A22EB595A70029B9C00CD
:109E00002A595378073B042B11D8D088FEF758FE07
:109E100000284ED0C3895A08D2182849029B0298BC
:109E2000CB542B5941180433254801F03DFD05B0B2
:109E3000F0BDFCF79FFD03000120834201D100200B
:109E40000393EB59DE88FCF79BFD03990200300079
:109E5000FFF7ECFB019AEB59117D042211420CD063
:109E6000217B114209D00B22C7E7F688FCF73CFDA5
:109E700001003000FFF7EEFB6BE7019A527D0121F4
:109E80000A4204D0607B084201D00C22B5E70221CF
:109E90000A4204D0607B084201D00E22ADE70421C3
:109EA0000A4204D0627B0A4201D01022A5E71222A6
:109EB000A3E7FA225200B0E75066FF1F5466FF1F67
:109EC0007FA2001110B5064B1A7804231000184029
:109ED0001A4200D00348FFF727FA002010BDC04601
:109EE000DD64FF1F8843FF1F70B50400FFF7D4FA3D
:109EF000051E43D12000FFF77FFA234EA400A0598E
:109F00008268937CDB0708D50321036A1B790B4029
:109F1000012B02D1017F0B430377431DD97F8B1E99
:109F2000022B0DD8022900D00121C088FCF790FF38
:109F3000042133591A7F59700A431A77280070BDDB
:109F400001290CD102231022437000210C3001F0B2
:109F500013FE305910213530FFF74BF9EEE7052994
:109F6000ECD10223D118437010220C3001F0ECFD2B
:109F700004233259117F0B431377EAE70825182889
:109F8000DCD1053DDAE7C0465066FF1FF0B58BB067
:109F9000059143887E4F9E00F45915000493002CD0
:109FA00015D1012902D000200BB0F0BD101D57784B
:109FB0001678FFF757F9EB68320002932B7A049971
:109FC000019300903B002000FCF70CFFEBE7E388D7
:109FD000049A934201D00820E6E72378012B00D1B0
:109FE000D4E0059B581E092800D9CFE001F08CFD74
:109FF00005CE0A29CC506C859AB229000498FFF747
:10A0000073FFD1E7200029001022453001F09CFDAC
:10A01000B9594B78042B02D1013B4B70C3E70B00BD
:10A020000A00253335320C310498FFF795F904986E
:10A03000FFF702FA0522431E9841BB59C0005A702F
:10A04000B2E7200029001022553001F07DFD049B6D
:10A050004F4C9D00295904980A0006AB55320C312B
:10A06000FFF77AF929591022453106A801F024FE9C
:10A07000012808D10498FFF7F7F90590002804D1CA
:10A0800006222B595A7005988EE708230593FAE7A4
:10A0900063780C2B7AD1E36E002B03D11C2001F0E6
:10A0A000D3FDE066BB59D86E00286FD0102229007E
:10A0B00001F04AFDBB590498DC6EFFF705FC0D2248
:10A0C000A076BB595A706EE7E06E00285ED06378C8
:10A0D0000D2B5BD12B8808220382A91C123001F0C2
:10A0E00033FDBB599A68517D0222114226D0186A6D
:10A0F000407B104222D00C32E4E763780E2B45D12E
:10A10000236F002B03D1162001F09EFD2067BB5961
:10A11000186F002803D01022290001F015FD0F222E
:10A12000BB59CFE763780F2B30D1206F0622691C13
:10A13000103001F009FDBB599A68517D042211428B
:10A1400003D0196A497B1142D5D100210498FFF749
:10A150008BFA28E7636F002B0DD0BB59586F00288E
:10A16000F3D01022290001F0EFFC0122BB5952422A
:10A170005B6F1A61E9E7142001F066FDBB59606767
:10A180005B6F002BE9D126E72978DFE707200BE793
:10A190005066FF1F10B5064C207001F015FB06211C
:10A1A0002078FDF791FF0348FEF778FC10BDC0460C
:10A1B0006366FF1F3593001100200BB270B50D00D0
:10A1C000834216DA264B187801F0D6FD041E0DD016
:10A1D0000378922B0ED0A02B37D0224B1878FF2873
:10A1E0003AD0210001F0A0FD002835D180200002E6
:10A1F000684070BD43780E2B0BD03E2BEDD1837899
:10A20000052B12D0082BE8D181798088FFF7D8FA86
:10A2100008E0154B82889A42DFD183681878591C70
:10A22000FEF7C0FE002817D1D7E7104B1B785B075D
:10A2300012D50F4B1B68002B0ED09B68002B0BD048
:10A24000C289811D80889847ECE7FFF741FAA06832
:10A25000002801D001F0C8FB200001F0D5FAC5E7C5
:10A260006366FF1F8143FF1F18200000DD64FF1F8E
:10A270004C66FF1F10B50078FFF712FA10BD10B53D
:10A280000078FFF7FDFA10BD0C234343084A10B5D0
:10A290009B185A68002A03D0012901D1904710BDAC
:10A2A0009B68002BFBD00029F9D19847F7E7C046FF
:10A2B0008066FF1F01238340094A10B5946B1C433D
:10A2C0009463506B98435063D46B200098430129EA
:10A2D00001D120001843D063116B0B43136310BDF1
:10A2E00000800040F0B500240127154B85B0DA6BE3
:10A2F000144E03921A6C0192DA64019BE3403B42D4
:10A3000017D0039DE5403D400295E5B20299280033
:10A31000FFF7BAFF316A736A002908D03900002BB1
:10A3200001D0029979402800FFF7C4FF01E0002B1B
:10A33000F9D101340C36172CDFD105B0F0BDC04681
:10A34000008000406466FF1F064B01215A68C2402E
:10A350000A4204D01B68C3401800084070471B6DB8
:10A36000F9E7C046008000400122064B82400029E8
:10A3700003D0D9680A43DA607047D9689143D9603D
:10A38000FAE7C0460038004030B5032444430F4B81
:10A39000E25C1B199C785D7801232D1B0135AB40D5
:10A3A000013BA340A140DB430C00122807D8084919
:10A3B00092005218116819402143116030BD054ABE
:10A3C00011680B4023431360F8E7C04637C0001103
:10A3D00008F0004014F00040C21F70B5D4B206234C
:10A3E000092C0BD80125084C9540002908D00021E4
:10A3F000FFF7CAFF23682B4323600023180070BDBA
:10A400002368AB43F8E7C04600380040214BF0B565
:10A410001B185B78022B21D1032444431E4A1F4E94
:10A42000A35C12199478012215008540B76B013C9A
:10A43000E4B23D43A240B563194C122815D89B00E5
:10A4400000290CD117495B1899680A439A600123C7
:10A45000205C154A834011680B431360F0BD11491D
:10A460005B18996891439960F1E70E4B00290DD173
:10A4700059690A435A61225C1328E8D00123203A23
:10A4800093400A49086803430B60E7E75969914321
:10A490005961F0E76466FF1F37C00011008000407B
:10A4A0007CC0001100F00040A0F00040A4F000408B
:10A4B000F8B500241B4E1C4D1C4B1B5D012B1FD1FE
:10A4C000194A9269E2401A420BD00122B2569340D7
:10A4D0002200143AD2B2022A09D815494A69134314
:10A4E0004B61013402360C35172CE5D1F8BD002242
:10A4F000B2560F499200521891680B439360F0E7EF
:10A50000022BEED1E7B23800FFF71EFF01235840BF
:10A51000C1B23800FFF77AFF3800FFF715FF687700
:10A52000DFE7C04609C000116466FF1F6566FF1FB4
:10A5300000F00040012202388240054B002903D080
:10A5400059690A435A617047596991435961FAE759
:10A5500000380040F8B50E0001210F008740114A75
:10A560000400D368FD43BB43D360831E8B4201D8F4
:10A57000FFF7E0FF00212000FFF72EFF0A4A0B4BF8
:10A580005168012E05D139431B1951605E700020BE
:10A59000F8BD2940516002221C1962709A69154069
:10A5A0009D61F4E700380040008000406466FF1FB2
:10A5B000012210B58240074B002906D019680A43D2
:10A5C0001A600121FFF7C6FF10BD19689143196099
:10A5D000F7E7C046008000400C2370B500254343D8
:10A5E0000A4A29009B181D70094B04001B185D7056
:10A5F000FFF7B0FF0123A340064928000A681A4369
:10A600000A6005490A689A430A6070BD8066FF1FA8
:10A610006466FF1F348000403080004070B5040045
:10A620000E00FF2813D003250540FFF7D5FF084A89
:10A63000A3089B009B183F22ED00AA40AE4019687A
:10A6400020009143314319600121FFF78DFE70BD59
:10A6500018380040F8B50C244443134B0500E418A7
:10A660006368002B03D1A3681220002B1AD00222AA
:10A6700001270E4B00215B195A7028002770FFF745
:10A6800069FF63681E1E08D0A3683E00002B04D03B
:10A690002800FFF759FE4640F6B228003100FFF7C8
:10A6A00009FE0020F8BDC0468066FF1F6466FF1FDC
:10A6B000F7B5C420FF222B4B80001958002491438A
:10A6C0003F3A0A431A508022274F5202274E1A60FF
:10A6D000274B1D5D002D21D0A31E012B03D8012186
:10A6E000E0B2FFF727FF012D18D11F4B9B69E34014
:10A6F0002B4213D0E3B218000193FFF725FE0100AF
:10A700000198FFF755FFE3B2143B022B1DD801213E
:10A710007156184A8D405369AB4353613B7F002B00
:10A720000DD0E5B22800FFF795FF2800FFF70CFEDB
:10A730007B7F0100834202D02800FFF7A5FD013492
:10A740000C370236172CC3D1F7BD012100237156F7
:10A75000F3568D40074A9B009B189A68AA439A605B
:10A76000DCE7C04600E100E06466FF1F09C000119D
:10A770006566FF1F00F0004070B50E001500040074
:10A78000FFF72AFF0C236343094A20009B189D60B2
:10A790005E60FFF75FFFF021064B074A8900051E48
:10A7A0005A5002D02000FFF717FF280070BDC046A6
:10A7B0008066FF1F0000FF1FE5A2001170B5134D5A
:10A7C00007202C78002C1FD198222100520028004D
:10A7D00000F0E2FF0123C420FF222B700C4B80000D
:10A7E0001C635C630B4B1C605C600B4B1958914302
:10A7F0003F3A0A431A50802252021A600D20074A3B
:10A80000074900F0A1FF200070BDC0466466FF1F2D
:10A8100000800040A0F0004000E100E0B1A600117F
:10A82000B1A40011030010B50620072B09D8054A72
:10A83000137001F089FAD7210020034B034A8900E5
:10A840005A5010BDB043FF1F0000FF1FCD1BFF1F5C
:10A8500070B51D0002240C2910D8094ACA40D2073D
:10A860000CD5FBF741FF041E08D1059A0499280076
:10A87000FBF756FFFCF7C4FDFFF724FB200070BD7B
:10A880001210000030B50D7802232C009C431842B2
:10A8900001D02B431C0008252300AB43284201D0E4
:10A8A0002B00234320241D00A543204201D01C433C
:10A8B00025002A230D70184204D011781E3B0B434B
:10A8C000137030BD0028FCD10C2113788B43F7E7BF
:10A8D000F8B51D0006AB1B88140007AA0E000B205C
:10A8E0001778002B27D10A78022A49D14A68507874
:10A8F00011780002244A08438018042840D801F047
:10A9000003F903121D1B2300F06801F055F8021C27
:10A91000C0B2B84200D93A1CD2B22000F1682A80F5
:10A9200001F012F906E00222F3681B882A802370E6
:10A930001B0A63700020F8BD0622EEE701232B807E
:10A94000F3681B782370F5E7F368002B16D0082214
:10A950002A801A8822701A88120A62705A88A27095
:10A960005A88120AE2709A8822719A88120A6271D1
:10A97000DA88A271DB881B0AE371DBE72B80D9E759
:10A9800001202B80D7E7C04600D6FFFFF7B51600A1
:10A990000A781D0008AB1F880C000123022A18D179
:10A9A0004A685078117800022B4A0843801803281F
:10A9B0000FD801F0A9F802254439E06800F0FCFF47
:10A9C000C0B20723B84204D37B190193152B02DDD3
:10A9D0000D231800FEBDE0682A003100C01901F007
:10A9E000B3F86B4600209B88E268D0541B4B1B6871
:10A9F000834203D01B68834200D098470023E8E7D6
:10AA00000B23002FE5D1022DE2D1737832781B029F
:10AA10001343E2681380114B1B68002BEED01B68B8
:10AA2000002BEBD00120E8E70B23002FD1D1062D1E
:10AA3000CED12A003100E06801F086F8DEE70B2372
:10AA4000002FC6D1012DC3D132787533012AC0D869
:10AA5000E3681A70D2E7C04600D6FFFF7068FF1F98
:10AA600070B50C001500072837D801F04DF8041414
:10AA700036361B36242E182015290BD8184E1622D0
:10AA80000021300001F078F822002900300001F0A8
:10AA90005BF8002070BD18200229FBD11288114BF1
:10AAA0001A80F6E718200829F4D10A000E48290078
:10AAB00000F02AFFEDE718200129EBD10B4B1078AD
:10AAC0000B49DA69FFF7DEFEE3E718200129E1D13F
:10AAD000064B10780749DA6BF4E70220DAE7C04644
:10AAE0005868FF1F2E44FF1F2444FF1FB443FF1F5D
:10AAF000DC43FF1FFC43FF1F030010B50020DB07F2
:10AB000004D50721024A034800F08CF810BDC04666
:10AB100094C00011B443FF1F054A030010680028C9
:10AB200003D082889A4201D1806870470068F6E7B6
:10AB3000686AFF1F0A88030008009A4204D08A88C6
:10AB400004309A4200D0002070470000F8B5F2228D
:10AB500000230D4F0D4E7968050042433370994232
:10AB600000D07B600A4C0021200001F005F8002392
:10AB70001A007C60AB4202D100203370F8BD013373
:10AB80002280DBB2F234F5E7606BFF1F5E6BFF1FC4
:10AB90006C6AFF1F73B56B4601900600684615008E
:10ABA0001980FCF75FFF041E11D1002D0FD07689AC
:10ABB000002E11D00C2001F047F800280ED0084AD2
:10ABC0000460136886808560002B02D1106020002D
:10ABD00076BD1A001B68F7E70224F8E71324F6E7AE
:10ABE000686AFF1F012100220A4B10B549420A4C36
:10ABF000198099809A719A70084B207001201980F1
:10AC00005A60FFF7A3FF2078FCF78AFF0448FDF79E
:10AC100045FF10BD7868FF1F686BFF1F606BFF1F4B
:10AC2000D1AC0011022310B5002802D0FFF7B2FF0B
:10AC30000300180010BD0000030010B50020DB0762
:10AC400004D50421024A0348FFF7A4FF10BDC04603
:10AC5000A8C000113444FF1FF0B50E2687B003933F
:10AC60000CAB1F8802ABF6180500080031000292F9
:10AC7000FDF77AF804000120002C0FD03088FFF790
:10AC80004BFF03000E20002B08D05E68002E05D07D
:10AC900021002800039B029A0097B04707B0F0BD3F
:10ACA0000A4B10B5984207D10122002352420A8074
:10ACB0008B708A808B7110BDFFF73CFF0028FAD0A3
:10ACC00001235B42038000238370F4E7FFFF000051
:10ACD000F8B5050001290AD1134E00243388F22764
:10ACE000AB4219D028001149FFF7DAFF06E002292C
:10ACF00004D10139FDF750FF0028EDD0F8BD3B002D
:10AD000063437268D018D35A002B09D03A0000214F
:10AD100000F032FF0134E4B2054B1B78A342EED8B9
:10AD200001235B423380DDE7606BFF1F7868FF1F04
:10AD30005E6BFF1F10B5FFF7FDFE0300002083428E
:10AD400000D0987810BD0000F0B589B01C000EABA3
:10AD500080CB03901E8810AB1B78049202930B7A71
:10AD60000D00DB0616D42B780593022B24D0049813
:10AD7000FFF7D2FE002812D003689C46002B0ED0AD
:10AD8000029B2200019329003B0064460398009631
:10AD9000A04705E00498FFF7BFFE002802D10E206F
:10ADA00009B0F0BD8368002BF9D00A22290003986E
:10ADB00098470028D7D0F3E76B6858781A786B4B20
:10ADC000000210439842D2D8043B984210D2684BFC
:10ADD000984242D015D8674BC0180128C7D80B201D
:10ADE000002EDDD1EB681A7859683A80200028E0FF
:10ADF000614BC018032800D979E000F085FE846A11
:10AE0000789E5E4B9842B2D10B20002EC8D1012310
:10AE10003B80EB6831001B7823706889013080B279
:10AE2000FCF7A2FF3A88031E0ED0017802328A187E
:10AE30003A80428962704289120AA2705968027887
:10AE4000E01C00F081FE06E004323A80310004226A
:10AE5000601C00F091FE0020A2E70B20002E9FD185
:10AE6000EB6807A91E8804233B80330A3000267054
:10AE70006370FCF779FF051E28D004AB9A890E2376
:10AE800004A95B183E49C668FCF7E2FF00280BD115
:10AE90002B783C486A680599FBF798FB002803D19A
:10AEA000012304AA5B42D3813278022A06D1716859
:10AEB000201D00F049FE3B8802333B800E2304AA8C
:10AEC0009B181B88A3701B0AE370C4E704ABDE81E8
:10AED000F4E70B20002E00D062E7E9680398FFF743
:10AEE00029FF02233B802070000A6070B3E70B202B
:10AEF000002E00D054E70222EB681B883A802370B2
:10AF00001B0A6370A7E7E86800F056FDC2B20300B1
:10AF10000720B24200D243E70DD00299DBB271188C
:10AF2000994202DB921BD3B20293029BE9681A009A
:10AF30003B8089195AE70023F6E70B20002E00D04A
:10AF40002EE70722EB683A801A7822705A786270EE
:10AF50005A88A2705A88120AE2701A792271DA8825
:10AF60006271DB881B0AA37175E7C04604290000E3
:10AF70000228000000D8FFFFFFD6FFFF03280000D3
:10AF8000FFFF0000D8BF0011F0B58DB06B46002068
:10AF9000089120229B5E83423DDAA64B187800F090
:10AFA000EBFE071E32D00378B02B2CD1007902388B
:10AFB00016281FD800F038FE17001E001E001E00C5
:10AFC00031001E0096001E001D011E0052011E00D1
:10AFD00073011E00CD011E0050021E001E001E0047
:10AFE0008E021E00E302944B94491B8878880B80E4
:10AFF000FBF72CF83800FCF7ADFF914B1B68002BDA
:10B0000001D038009847380000F0FEFB8020089BF4
:10B010000002434018000DB0F0BDEE220021874829
:10B0200000F0AAFD0BAA3B7B7989388900923A008F
:10B030000D32FCF7B1FD0400804B1B78002C3FD192
:10B0400046E0804B788805937F4B4100CB5A0BAE8E
:10B05000073BDBB232880293002301937B4B210034
:10B0600006930093059BFFF76FFE744D002810D1E7
:10B07000069B3A8A1B889A420BD1380005991230F8
:10B0800000F01AFE002804D02B7862899B00EB1890
:10B090005A80162306A81B18328820007989FCF7ED
:10B0A000D7FE2B7804009A00AA1851880029C3D033
:10B0B0000133DBB22B70002807D006A9C98A918022
:10B0C000634A12889A42BCD802E001214942918029
:10B0D000002B04D059497888FAF7ECFF8AE73E89BB
:10B0E0000A2479E000253E89574B06937B88069A0F
:10B0F0005B009B5A033B9D4202DB002DF0D05BE0DE
:10B10000162206A812183B7B798900923A0030007B
:10B110000D32FCF741FD0590002858D04689017A90
:10B120007888FCF703FD041E44D1464B78880793CA
:10B13000069B4100C95A454B0439C9B206AAD28AB6
:10B1400006930291019400930599079BFFF7FCFD7C
:10B15000041E2FD1069B39491A88931C002D26D135
:10B160004B807988384B4900CB5A5119033B8B42AD
:10B1700020DD059B31485B8941190B71A91C013504
:10B18000C9B2EDB2059145191B0A2B71059B2D49DA
:10B190000433181800F0D8FC2C4B059A1B88D318E0
:10B1A000DDB22C4B9E4205D00136B6B29CE74988F1
:10B1B0009942D6D0002D0CD0204C2800618800F098
:10B1C0007BFC207021007888FAF784FF12E7059C49
:10B1D000F0E7002C00D183E77B78142B00D109E73E
:10B1E00016493B794E800B700C717888FAF724FF72
:10B1F00000E7162406ABE41821003889FCF7B4FDFB
:10B20000011E00D1B7E1788822880F4C45002C5BE5
:10B210000A4D013CE4B2029400240F4B01940095C6
:10B22000FFF792FD041E00D014E129007888FAF798
:10B2300061FFDFE6686BFF1F2043FF1F8068FF1F71
:10B240007468FF1F7469FF1FB064FF1F646AFF1FEB
:10B250001E43FF1FFFFF00008268FF1F162406AB7E
:10B26000E41821003889FCF77FFD011E00D182E13E
:10B2700078882288AE4C45002C5BAE4D013CE4B290
:10B2800002947C89AC4B01940095FFF75DFD041E90
:10B2900000D0DFE029007888FAF736FFAAE600251B
:10B2A000A44B1D803B00F6331B78A24A7888079296
:10B2B000AB4208D99E4B12880693069943005B5A0D
:10B2C000013B9A4203DB0799FAF728FF92E616241E
:10B2D0006B00FB18059306ABE418059B2100188949
:10B2E000FCF742FD011E03D1059B01241E8973E773
:10B2F0007888924B2288069C099343001B5B904EF2
:10B30000013BDBB20293002300960193099BFFF7F8
:10B310001BFD041E02D0059B1E895DE77B88069AF3
:10B320005B009B5A079A108832881218934202DCFD
:10B330001B1A013B33807F4C023032880999001977
:10B3400000F002FC2388328801359B182380EDB27F
:10B35000A8E70BAA3B7B7989388900923A000D3225
:10B36000FCF71AFC00250590059B002B04D10A244C
:10B37000002D00D16EE060E0059B7888197AFCF71B
:10B38000D5FB0100041E63D1694C6C4B7888069490
:10B390000993069B4400E45A694B063CE4B20BAEA9
:10B3A000328807930294019100930599099BFFF756
:10B3B000CBFC041E4CD1079B5E491B881A1D002D37
:10B3C00030D14A80059B5B4C5A8963191A716B1CFA
:10B3D0009BB2E318120A1A71162306A832881B18AA
:10B3E00079890598FCF734FDFF21AA1C2E1D033531
:10B3F0000B00059092B2B6B2ADB2002803D006ABF6
:10B40000DB8AD9B21B0AA218651911712B714C4D38
:10B41000301D2A884949201800F096FB2B88F61821
:10B42000B5B2A1E74988914207D17A8806995200BE
:10B43000525AEB18053A9A42C4DC3E4C2800618807
:10B4400000F062FC207021007888FAF771FED1E5E7
:10B45000002DF2D13E89BFE6162606ABF618310064
:10B460003889FCF781FC3D000400FA3500282DD016
:10B47000037A9B060CD400227B8939897888009254
:10B480003A000C32FFF7E8FB041E10D03E8915E0AD
:10B490003088FFF741FB00281AD08368002B17D0B3
:10B4A0002100122278889847041EE4D0EEE72B781A
:10B4B000002B02D17888FAF74BFE00262B78002B60
:10B4C00000D097E5002C00D194E585E60124DDE766
:10B4D0000E24DBE7162506ABED1829003889FCF7AA
:10B4E00043FC041E47D0037A9B0611D4154A7B887F
:10B4F0001188994203D01448814207D11380134B1D
:10B50000F2261D780023D9B2A94221D30924A1E74C
:10B510002888FFF701FB00282FD08368002B2CD050
:10B520002100122278889847041EDFD092E7C04697
:10B53000B064FF1F8068FF1F8268FF1F7469FF1FD0
:10B54000646AFF1F606BFF1FFFFF00005E6BFF1F41
:10B5500031005943546801336018615A0029D2D12F
:10B560003C0008342100F22200F0EEFA2100788835
:10B57000FAF7F6FD3EE501246CE70E246AE71D4B61
:10B580001A887B889A4231D07888FAF7F3FD31E542
:10B59000F223059851684343CD18C95A00291FD09A
:10B5A0003B7A012B0BD16C88AB887888AA1D00945C
:10B5B000FFF752FB041E02D000233B722E88F222BA
:10B5C0000021280000F0D8FA00232B80059B0133CE
:10B5D000DBB20593084B05991B78064A8B42D7D8F6
:10B5E00001235B421380002CCED0F5E50026340009
:10B5F0000596EFE7606BFF1F5E6BFF1F70B50400E1
:10B600000E001500FFF796FA031E08D13100054819
:10B61000FFF790FA03001120002B02D01C800020BD
:10B620009D7070BDFFFF0000F8B50B4F06003B7822
:10B630000D001400FF2B0ED00A2000F08DFB011E20
:10B6400009D0B1230380002346800371C5800481A3
:10B65000387800F069FBF8BD7544FF1FF7B50F009F
:10B6600008A90600088809A90B240988002821D107
:10B670000234022B1ED1557813782D021D432B0066
:10B680008B4301937334002B14D1FB6830001900F5
:10B690000093FFF74FFB019C85420BD02A0030003E
:10B6A0000099FFF7ABFF041E04D12A00300079890E
:10B6B000FFF7BAFF2000FEBDF0B50E7885B003900D
:10B6C0000AA805880120022E0DD14C6827786478DD
:10B6D00024023C43054FBC4205D10398DBB20196DE
:10B6E0000095FFF7BBFF05B0F0BDC0460229000082
:10B6F000034B10B51B68002B00D09847FEE7C046EF
:10B700006C6BFF1F07B501A8FFF7F2FF044A05485D
:10B710000021121A00F040F8F8F7AEF8FEE7C04634
:10B72000706BFF1F7844FF1F01B40248844601BCC0
:10B73000604700BF6571010001B40248844601BC46
:10B74000604700BFC56D010001B40248844601BCDA
:10B75000604700BF4D31FF1F01B40248844601BC61
:10B76000604700BF014C010001B40248844601BC9F
:10B77000604700BF1147010001B40248844601BC84
:10B78000604700BFE548000001B40248844601BCA0
:10B79000604700BF5139FF1F01B40248844601BC15
:10B7A000604700BFB70E000001B40248844601BCE8
:10B7B000604700BF3D39FF1F01B40248844601BC09
:10B7C000604700BFC521000001B40248844601BCA7
:10B7D000604700BFC926000001B40248844601BC8E
:10B7E000604700BF5549010001B40248844601BCCE
:10B7F000604700BF456B010001B40248844601BCAC
:10B80000604700BF613BFF1F01B40248844601BC92
:10B81000604700BF434D010001B40248844601BCAB
:10B82000604700BF2D33FF1F01B40248844601BCAE
:10B83000604700BF9536FF1F01B40248844601BC33
:10B84000604700BF8D12000001B40248844601BC6D
:10B85000604700BF5D17000001B40248844601BC88
:10B86000604700BF6D2EFF1F01B40248844601BC33
:10B87000604700BFE928000001B40248844601BCCB
:10B88000604700BF5D34FF1F01B40248844601BC1D
:10B89000604700BFED32FF1F01B40248844601BC7F
:10B8A000604700BF453BFF1F01B40248844601BC0E
:10B8B000604700BFA946010001B40248844601BCAC
:10B8C000604700BF0919FF1F01B40248844601BC4C
:10B8D000604700BF3519FF1F01B40248844601BC10
:10B8E000604700BFC530FF1F01B40248844601BC59
:10B8F000604700BFF30E000001B40248844601BC5B
:10B90000604700BF350E000001B40248844601BC08
:10B91000604700BF810E000001B40248844601BCAC
:10B92000604700BF311B000001B40248844601BCDF
:10B93000604700BF8552010001B40248844601BC43
:10B94000604700BF1D4B010001B40248844601BCA2
:10B95000604700BF4551010001B40248844601BC64
:10B96000604700BF2146010001B40248844601BC83
:10B97000604700BFC9A9000001B40248844601BC69
:10B98000604700BF291C000001B40248844601BC86
:10B99000604700BF5125000001B40248844601BC45
:10B9A000604700BFA136FF1F01B40248844601BCB6
:10B9B000604700BF753AFF1F01B40248844601BCCE
:10B9C000604700BFDD52010001B40248844601BC5B
:10B9D000604700BF2951010001B40248844601BC00
:10B9E000604700BF8B52010001B40248844601BC8D
:10B9F000604700BFD949010001B40248844601BC38
:10BA0000604700BFF13AFF1F01B40248844601BC01
:10BA1000604700BF5147010001B40248844601BCA1
:10BA2000604700BFB14E000001B40248844601BC2B
:10BA3000604700BF3555000001B40248844601BC90
:10BA4000604700BF691F000001B40248844601BC82
:10BA5000604700BFA54F010001B40248844601BC05
:10BA6000604700BF156B010001B40248844601BC69
:10BA7000604700BF0124000001B40248844601BCB5
:10BA8000604700BFD91B000001B40248844601BCD6
:10BA9000604700BFB54C010001B40248844601BCB8
:10BAA000604700BF090E000001B40248844601BC93
:10BAB000604700BF851F000001B40248844601BCF6
:10BAC000604700BF350E000001B40248844601BC47
:10BAD000604700BFC94A010001B40248844601BC66
:10BAE000604700BFB352010001B40248844601BC64
:10BAF000604700BFDD66010001B40248844601BC16
:10BB0000604700BFE117000001B40248844601BC51
:10BB1000604700BF753BFF1F01B40248844601BC6B
:10BB2000604700BF75A9000001B40248844601BC0B
:10BB3000604700BF4D1F000001B40248844601BCAD
:10BB4000604700BF093AFF1F01B40248844601BCA8
:10BB5000604700BFE94C010001B40248844601BCC3
:10BB6000604700BFAD30FF1F01B40248844601BCEE
:10BB7000604700BFEDA5000001B40248844601BC47
:10BB8000604700BF154D010001B40248844601BC66
:10BB9000604700BF5952010001B40248844601BC0D
:10BBA000604700BF017F000001B40248844601BC29
:10BBB000604700BF4938FF1F01B40248844601BCFA
:10BBC000604700BF2124000001B40248844601BC44
:10BBD000604700BF7918000001B40248844601BCE8
:10BBE000604700BF5522000001B40248844601BCF2
:10BBF000604700BF091B000001B40248844601BC35
:10BC0000604700BFC536FF1F01B40248844601BC2F
:10BC1000604700BF1D3BFF1F01B40248844601BCC2
:10BC2000604700BF2526000001B40248844601BCDD
:10BC3000604700BF893BFF1F01B40248844601BC36
:10BC4000604700BFF94C010001B40248844601BCC2
:10BC5000604700BF3D4B010001B40248844601BC6F
:10BC6000604700BF6DBC000001B40248844601BCBF
:10BC7000604700BF9537FF1F01B40248844601BCEE
:10BC8000604700BFC939FF1F01B40248844601BCA8
:10BC9000604700BFADAE000001B40248844601BC5D
:10BCA000604700BF0D52010001B40248844601BC48
:10BCB000604700BF056A000001B40248844601BC29
:10BCC000604700BFCD4C010001B40248844601BC6E
:10BCD000604700BF3D18000001B40248844601BC23
:10BCE000604700BF9DA9000001B40248844601BC22
:10BCF000604700BFC51D000001B40248844601BC76
:10BD0000604700BF4550000001B40248844601BCB2
:10BD1000604700BF090E000001B40248844601BC20
:10BD2000604700BF055E000001B40248844601BCC4
:10BD3000604700BF594F010001B40248844601BC6E
:10BD4000604700BF8939FF1F01B40248844601BC27
:10BD5000604700BFCD1BFF1F01B40248844601BCF1
:10BD6000604700BF1D4D010001B40248844601BC7C
:10BD7000604700BFED4A010001B40248844601BC9F
:10BD8000604700BFF54E010001B40248844601BC83
:08BD9000604700BFFD19FF1F11
:10BD9800000301020203030304030500060207006F
:10BDA800080209030A030B030C000D000E030F031E
:10BDB8001003110313031403150216023D3C00116E
:10BDC800713C00110000000002000000DABD001103
:10BDD800192A0F180A000000F1590000FD2400007C
:10BDE80041460100A5810011B9A100110D7600118D
:10BDF800A97F00115154001189AF00119D50001105
:10BE08004D3E00117D3F0011000000001616000095
:10BE18000200000024BE0011F4FFF3FFD2FC000072
:10BE2800BD40001100000000000000005475796159
:10BE38000042322E30003030314100676974687535
:10BE4800622E636F6D2F7076767800544842330007
:10BE5800020000006CBE0011292A282A272A262A57
:10BE6800252A242A0A180000E204000071020000B2
:10BE780078EC000005000000744000001027000066
:10BE880060F000000400000006640000204E00007E
:10BE980000000000060000005C44000010270000BD
:10BEA8006CEE000007000000050000001F501D1088
:10BEB800023CB40000011A0020000000A1020000AA
:10BEC80030313233343536373839414243444546C8
:10BED8000000000055580011A9580011000000008A
:10BEE80002000000F4BE00116F2A6E2A1A18EAD860
:10BEF800BC80F0FC600000000000000000005F064D
:10BF08006B2F363D7D077F3F777C596E7971000036
:10BF180001A00000000000006410B71DC8206E3B9F
:10BF2800AC30D9269041DC76F4516B6B5861B24D38
:10BF38003C7105502083B8ED44930FF0E8A3D6D6A2
:10BF48008CB361CBB0C2649BD4D2D38678E20AA00A
:10BF58001CF2BDBDFB349B5F800000800010000018
:10BF6800000000000F62001199780011336200117F
:10BF7800A17C0011B7620011777C00112D630011BC
:10BF88004D7C00117F630011157E0011E7630011DD
:10BF9800157E001119640011CF7D00112D63001169
:10BFA800057C0011A5630011AD7D001100000000A3
:10BFB800000000008B640011AD7D0011ED640011DC
:10BFC800B1780011052A042A012A002A0229032827
:10BFD80001280028011800180000000000000000D7
:10BFE80000000000000000870101020102010102B7
:10BFF800010203030401030101010101030302011A
:10C0080003000D000E0010001100130014010701B9
:10C0180008010A010B011C011D02040205020702A6
:10C02800080219021A021C021D0301030203170069
:10C038000201000504000807000B0A001716001D7E
:10C048001C010201010504010E0D01111001141358
:10C05800011716011A19020201020B0A020E0D023B
:10C068001110021413021716030504030807030B23
:10C078000A030E0D0001020307090A0B0E0F101127
:10C0880012141718191A1B1F20212200D1A80011F9
:10C098008DA900110000000002000000DEBF0011A1
:10C0A80000000000B9B60011000000000200000006
:04C0B800DCBF0011D8
:020000041FFFDC
:1000000000000000B53D0011E0BD0011DCBD001195
:10001000A861FF1F000000000000000000000000B9
:1000200000000000000000000000000000000000D0
:1000300000000000000000000000000000000000C0
:1000400000000000000000000000000000000000B0
:1000500000000000000000000000000000000000A0
:100060000000000000000000000000000000000090
:100070000000000000000000000000000000000080
:100080000000000000000000000000000000000070
:100090000000000000000000000000000000000060
:1000A0000000000000000000000000000000000050
:1000B0000000000000000000000000000000000040
:1000C0000000000000000000000000000000000030
:1000D0000000000000000000000000000000000020
:1000E0000000000000000000000000000000000010
:1000F0000000000000000000000000000000000000
:1001000000000000000000000000000000000000EF
:1001100000000000000000000000000000000000DF
:1001200000000000000000000000000000000000CF
:1001300000000000000000000000000000000000BF
:1001400000000000000000000000000000000000AF
:10015000000000000000000000000000000000009F
:10016000000000000000000000000000000000008F
:10017000000000000000000000000000000000007F
:10018000000000000000000000000000000000006F
:100190005133FF1F9931FF1FC166010000000000AD
:1001A000000000000000000000000000000000004F
:1001B000000000000000000000000000000000003F
:1001C000000000000000000000000000000000002F
:1001D000000000000000000000000000000000001F
:1001E000000000000000000000000000000000000F
:1001F00000000000000000000000000000000000FF
:1002000000000000000000000000000000000000EE
:1002100000000000000000000000000000000000DE
:1002200000000000000000000000000000000000CE
:1002300000000000000000000000000000000000BE
:1002400000000000000000000000000000000000AE
:10025000000000000000000000000000000000009E
:10026000000000000000000000000000000000008E
:10027000000000000000000000000000000000007E
:10028000000000000000000000000000000000006E
:10029000000000000000000000000000000000005E
:1002A000000000000000000000000000000000004E
:1002B000000000000000000000000000000000003E
:1002C000000000000000000000000000000000002E
:1002D000000000000000000000000000000000001E
:1002E000000000000000000000000000000000000E
:1002F00000000000000000000000000000000000FE
:1003000000000000000000000000000000000000ED
:1003100000000000000000000000000000000000DD
:1003200000000000000000000000000000000000CD
:1003300000000000000000000000000000000000BD
:1003400000000000000000000000000000000000AD
:10035000000000000000000000000000000000009D
:10036000000000000000000000000000000000008D
:1003700005B70011000000000000000000000000B0
:10038000000000000000000000000000000000006D
:10039000000000000000000000000000000000005D
:1003A0000000000000000000000000004D1BFF1FC7
:1003B000000000000000000000000000000000003D
:1003C000000000000000000000000000000000002D
:1003D000000000000000000000000000000000001D
:1003E000000000000000000000000000000000000D
:1003F00000000000000000000000000000000000FD
:08183800706FFF1F4118FF1F34
:10184000024981F3088802F0CBFB0000706FFF1F94
:1018500070B500241E491F4A1F484C6308CA1B0567
:101860001B0DE4188242F9D11C4B80228B630021AE
:1018700009201B4B920519621A4B1B4DDA671B4B53
:10188000DA688243DA609A68194802409A60112047
:10189000296002F0B9F8112002F096F86B6C154A35
:1018A000112013406B64EE23DB006343124A1B0CD0
:1018B00013840122114B9A7201F024FC104B1B7807
:1018C000002B04D10F4B1021187802F0B9F970BD2C
:1018D000000005400806054080060540FF010000A5
:1018E00000F0004004E100E0003800403CF000401F
:1018F000FFDFFFFFFFFEFFFF7861FF1F2C62FF1F6E
:101900005A64FF1F5862FF1F10B502F091FB0728B1
:1019100004D0122808D0022808D010BD044A0420A0
:10192000136B01331363F8E70220F6E71420F4E7A2
:101930005865FF1FF8B507000C002600250050363B
:1019400030785135002804D10300287058342370B2
:10195000F8BD2978CA00481E8141A3183800A25C4E
:101960005B68C9B2FFF7D0FF00280DD12B78DA00F1
:10197000A218013350602B703378044A013B337056
:10198000136A01331362D8E70123DFE75865FF1FAD
:101990005C234343074910B5C9180B0058331B7823
:1019A000012B05D1FFF7C6FF034A936A0133936207
:1019B00010BDC0468C65FF1F5865FF1F10B502F0B3
:1019C000A7F9064A0121130010CB4942D967044BFD
:1019D000136002F025FB200010BDC04600E100E0CE
:1019E0001000100010B5040002F092F9024B1C60C8
:1019F00002F016FB10BDC04600E100E010B5040087
:101A000002F086F94021094A200013688B431360D5
:101A100000F0F6FA01F07EFC0022054B01201A606E
:101A2000044B04321A6002F02BF9FEE71CF0004070
:101A3000C4F00040C0F00040431E5A425341A0226F
:101A4000F0B5D2015B421340154D164A40019B1878
:101A50002A18127E8BB00191002A1BD01A0008327E
:101A6000D46F0022E6B206AFE4B294420EDC28182E
:101A7000C369002B08D0019902AA117106AA049229
:101A800002AA167303A898470BB0F0BD1978B95491
:101A90000132EAE71A7D1A7806AB01261A70E6E7EA
:101AA0001868FF1F00400040F0B5254B04004001BE
:101AB000C25C85B0002A2BD01A18117E002927D0CD
:101AC000917E002924D01179022921D11689D78845
:101AD000D168F51BADB22A1C102D00D9102292B28C
:101AE000BE4217D11818012303710023C269C380B5
:101AF00003819A4206D06846032103730171029361
:101B000001A890470820002C00D0192001F0FAFA13
:101B100005B0F0BD013C65426C41A0256442ED0179
:101B20002C40084D1B186419074D0633013A92B238
:101B3000AA42EDD01888461C1E80085C2070F5E78C
:101B40001868FF1F00400040FFFF00000F220E4BEF
:101B500010B59868104002380A280BD802F00AF82D
:101B60000D0A0B0A0A110A0A0A0A060002210020BD
:101B7000FFF762FF10BD0121F9E70020FFF794FF96
:101B8000F8E7DB6FF6E7C046004000400F220E4B3F
:101B900010B59868104002380A280BD801F0EAFF07
:101BA0000E0A0B0A0A120A0A0A0A0600022101207A
:101BB000FFF742FF10BD01210800F9E70120FFF700
:101BC00073FFF7E7DB6FF5E70090004013B5334C88
:101BD0002378072B3DD8324B1A78324B002A39D163
:101BE0008022196852020A431A60252001F0CCFEB7
:101BF00020232D4A11680B43802113606B46042279
:101C0000C90508680733104228D080210422C9057D
:101C1000C86810422ED080212020C905CA6882439E
:101C2000CA6014221A701A78002A2FD18021C9059F
:101C3000C86820320243CA6014221A701A78002A37
:101C400028D11A4B1A7D22785A601D221A705932F7
:101C5000DA6013BD1A6816490A40C5E708680243EE
:101C60000A6014221A701A78002ACED01A78013A23
:101C7000D2B2F7E7C8680243CA6014221A70197812
:101C80004A1ED2B21A700029F9D1C4E71A78013A73
:101C9000D2B2C7E71A78013AD2B2CEE7B043FF1FFB
:101CA0007844FF1F3CF00040A843FF1F0020004085
:101CB000FFFFFEFF564B70B51B68012B03D1554A41
:101CC000936D0133936502F01BF9534B534A18602F
:101CD000534B544C1A600123534A1360534A136008
:101CE0002378002B06D006225149524802F010F901
:101CF00000232370504A514B10681B78C1B2002B4F
:101D00000ED14F4CC0B223785BB2002B4FDB23784F
:101D100024785BB264B21B0424021B191B181360E5
:101D20000B1C50294ED95023464A47491078DBB244
:101D3000FF2202284BD10868444C454D2678904339
:101D40002A78964254D9227824782E78023B5D1066
:101D5000A31B6B435201D31A10335B111843086065
:101D600002F096F8031F012B45D83A4B1B78002B45
:101D700006D0394B1B78002B02D0002002F030F83F
:101D8000A122364B92009978354B4A431B689B1829
:101D9000832292009B181B78033B012B03D8AF20B2
:101DA000400002F02DF901222E4BDA8270BD23781B
:101DB00024785BB264B2FF33FF341B0424021B1986
:101DC0000138ABE7CAB2022AAED20223ACE70868F8
:101DD000254C264D267890432A78964208D92278B9
:101DE00024782D78023B5B10641B63435201B2E7F9
:101DF0002378DBB2B2E70228D5D11D4B1B78013B1B
:101E0000022B03D91B4B1B78022BCCD16C20C8E7CB
:101E10009809FF1FFC0FFF1FA464FF1FFF3F000076
:101E200014100340A864FF1F0C100340001003406F
:101E3000D50BFF1F7211FF1FB40003408C09FF1F59
:101E4000680AFF1F490AFF1F94000340460AFF1F4C
:101E5000470AFF1FF908FF1F2209FF1F300DFF1F50
:101E60003409FF1FBC0BFF1F440AFF1F450AFF1F59
:101E70001C09FF1F2309FF1F10B501F099FE002266
:101E8000014B1A8010BDC046A264FF1F10B502F0BE
:101E90000FF8A121054A89009478054A6143126828
:101EA000044B5218528C1A8010BDC046300DFF1FD3
:101EB0003409FF1FA264FF1F10B50D4B0D4A99781E
:101EC000A1239B004B431268D218531DD97F0A4BA4
:101ED0001B88994209D2441C07D0C82805D0D26972
:101EE0005B1A5A43054B5343C01801F099FF10BDCC
:101EF000300DFF1F3409FF1FA264FF1F7102000095
:101F000070B5244D2B68002B28D001F0E9FF2B6819
:101F1000D8402B680400002B27D001F061FE2B680D
:101F2000D8401D4B1D4A9978A1239B004B43126852
:101F3000D118D25C91239B00002A20D0CA580132CC
:101F4000CA50174B17491B680868834214D3D23B09
:101F5000181A012A1AD0144B186070BD01F0C0FF86
:101F6000124B196801F0E4FFD3E701F039FE0F4B83
:101F7000196801F0DDFFD4E70D495B18E8E7CA50A6
:101F80000C4B1B68DB68E418201AE4E7F530FF30DF
:101F9000E1E7C0461C08FF1F300DFF1F3409FF1F7B
:101FA0009C09FF1FA464FF1FA009FF1F1808FF1F43
:101FB0002DFF3F00AC64FF1F70B504000D00282901
:101FC00016D10300A433C2881B889B1A0B4A9BB20C
:101FD00093420DD906006A3605223100653001F0C2
:101FE000F7FF002804D13100200001F0F1FE70BDA0
:101FF0002900200001F034FEF9E7C046FE7F000012
:10200000F8B50500012001F013FE134CA36AA26A83
:102010009342FBD1114E336001F04AFE1049030098
:1020200008601048426894460F4A17680022BC4571
:1020300001D24268BA1A0D4802603268AD18A42273
:10204000E562606A520302436262094A1278002A1A
:1020500001D00F3B0B60F8BD00F00040340AFF1FB9
:10206000E408FF1F28100040180AFF1F1C0AFF1F6A
:102070001C09FF1F70B580241025E405A3682B43BD
:10208000A36001F05DFEA368AB43A36070BD0000D8
:10209000F7B5160080221C001023D205019191682B
:1020A00005000B43936000225A4BD7301A6001F0B1
:1020B00047FF9D232A002F009B00EB58CA320121C5
:1020C0000092FC37002B01D00021009A386801F003
:1020D000E7FF2900009BCB311A784F4BD3351A60AC
:1020E0004B780A781B0213438A7812041A43CB7880
:1020F0001B061343494A1BBA13604B790A791B022A
:1021000013438A7912041A43CB7931001B06134317
:10211000434A1BBA13606B782A781B021343AA78D0
:1021200012041A43EB781B0613433E4A1BBA136092
:10213000019A330213433C4A13603C4B22001B1BA1
:102140009C4603293DDCB3089A0013005142B21AA1
:10215000032A46D1354AE018511A82784078120491
:1021600000020243E05C043302430A600022FF2BBA
:102170004BDDF0222E4B12011A600F222D4B1A60FC
:102180002D4A1368002BFCD00023224A27491360F4
:10219000091B321D0B191B68043A180A2370607062
:1021A000180C1B0EA070E3700434002AF2DC8022AD
:1021B00010213B68D20501333B6093688B439360E9
:1021C000F7BD6346D578981893782D061B042B43EA
:1021D000157804392B43557804322D022B430360C4
:1021E000AFE7022A0AD1114AE05C511AE21852788C
:1021F000120202430A6004339BB2B7E7012AB5D149
:102200000A4A521AE15C1160F5E7084959180A6058
:102210000433ACE7000004403C00044038000440B4
:1022200034000440300004400C000440000104402D
:10223000040004401000044014000440F7B51500E9
:1022400080221C001023D2050091916807000B43E7
:1022500093600023654AD730136001F071FE9D231F
:102260003E009B00F9583B00CA363200FC3300297F
:1022700000D07FE0586801F013FF390032785C4BE2
:10228000CB311A604B780A781B0213438A78AC462C
:1022900012041A43CB78281D1B061343554A1BBA58
:1022A00013604B790A791B0213438A7912041A438B
:1022B000CB791B061343504A1BBA13604B7A0A7A38
:1022C0001B0213438A7A12041A43CB7A21001B069D
:1022D00013434A4A1BBA1360009A2B021343484A1D
:1022E00013602200474B1B1B0093009BCE785B18AA
:1022F00001938B7836061B0433430E78043833433E
:102300004E78043136023343019E33600328ECDCFF
:102310000321A808431C9B002940800003292BD1DE
:102320003849E5185E18A9786D78E35C09042D0238
:10233000294319433160030008330021FF2B2DDDB1
:10234000314B324919600F21314B19600123274964
:102350000B60304B19680029FCD006211B680B402C
:10236000042B20D080220020D20593680A318B43B1
:102370009360FEBD01217DE7022908D121495D1846
:10238000E1184978E35C090219432960D3E7012980
:10239000D3D11C495918E35C0B60CCE719481818D5
:1023A00001600433CAE7002310490B606346002B29
:1023B0000CDC3B00FC335A68102101325A60802249
:1023C000D205936801208B439360D2E7009B9B1852
:1023D0001B68190A13705170190C1B0ED37004235B
:1023E0005B4291709C440432E0E7C0460000044028
:1023F0003C000440380004403400044030000440F5
:102400000C0004400001044004000440080F0000D8
:10241000100004401400044070B5061E19D00222BA
:102420005A4B9B799343012B13D1594B1A78FF2AAE
:102430000FD15A78FF2A0CD19A78FF2A09D1DA787D
:10244000FF2A06D11A79FF2A03D15B79FF2B00D12D
:1024500099E0504B0C201A78012A08D000224E4DEA
:102460001A7029780B00093B042B01D8212070BD7C
:102470004B1F012BFAD9454CA37B042B00D982E0DA
:10248000A279032A00D97EE09A1ED2B2012A02D88C
:1024900060881F2877D9002E56D0012E73D1A088CE
:1024A0000128E3D0002907D1581E032803D801F0E2
:1024B00061FB121715122E702978481E032811D8B7
:1024C0000025364B1D602823237501F0E1FBA8424F
:1024D00027D0A580CAE702212970EDE70421FBE798
:1024E0000321F9E707390129C0D82D490968C96ACC
:1024F0008906BBD52B4908780028B7D1012A01D914
:10250000002BB3D102230B708021274D2633890184
:102510002878237501F08CFC80212878890101F04E
:102520008FFB0123A380214B1B78002B0AD0FA22BA
:1025300080211F4B92001B8809025A431A4B1878BE
:1025400001F0AEFB002092E701F0E2FB2B78A680C1
:10255000073B012B03D917482E7001F0B1FC114B3A
:10256000114C1A78002A06D0802100222078890197
:102570001A7001F05DFC01F053FD80212078090202
:1025800001F056FCDEE7122071E7C046A60BFF1FE4
:102590006B09FF1F1A09FF1F1C09FF1F4809FF1FB6
:1025A000AC64FF1F2309FF1F1B09FF1F2109FF1F29
:1025B0002C09FF1F0010004010B5002901D001F0C8
:1025C0003FFC10BDF7B5604B01919978A1239B00AA
:1025D0004B435E4A060014681022E418D6235B00C1
:1025E000E0583623FF33E35C00279343222B41D18D
:1025F000574B0F3A1A600760012501F0B9FB019BA8
:102600001880E8235B00E35C002B01D0B34258DD67
:102610000023504FFB70AD33FF33E3581A68002A94
:1026200003D09B88DB439B071DD03823FF33E35C3B
:10263000002B18D09B235B00E35C002B13D1D1331C
:10264000FF33E35CB3420EDAA4235B00E15AE018E7
:10265000090A023101F084FB23000122FE33013E0E
:1026600001351A87FA70E8235B00E35C002B2AD05F
:10267000A8B2FEBD03683D00002BBED081880430A7
:10268000090A023101F06CFBD6235B00E3581F609E
:10269000B2E72300B133BA00FF339858013781887D
:1026A0000430090A023101F05BFBE8235B00E35CC4
:1026B000BB42EEDCE822F61AED1800235200A354C8
:1026C000A6E70027F1E7200001F09AFB00281FD0C1
:1026D000002E1DDD7319882647190193B6002000CE
:1026E00001F006FB5A3080002018406801358188CF
:1026F0000430090A023101F033FB200001F048FBED
:10270000A3590133A351BD4202D0019B9D42E6D1A2
:10271000114BE35C002BABD095239B00E35C002BBB
:10272000A6D00E4BE15A0029A2D00D4AA35C9942D3
:1027300002D90133A3549BE700231A212000A3549C
:1027400001F086FA94E7C046300DFF1F3409FF1FE1
:1027500000140340E010FF1F5A0200007202000044
:102760005E0200000D4970B54A6E0D4CD2038B69B4
:10277000D20BA24206D80B4D0224AA4204D901F082
:10278000FFFA70BD02246442E21815007E24254041
:102790002242F4D0A3432B438B61F0E700F00040CA
:1027A0000A200000FC1C0000F8B51D4B1D4F1A78D4
:1027B000002A10D1BA7B002A02D101321A7003E03C
:1027C000032AFAD0022AF8D001F062FA002201208E
:1027D000154B1A70F8BD154B154D1C68154B9E789E
:1027E00001232B702878C0B200F09EFBBB7B002B2E
:1027F0000BD101F0B5FBA1239B007343E4188323A5
:102800009B00E41823782B70E4E7032B02D101F03E
:1028100087FAF0E70020022BDCD101F061FAEAE749
:102820001C09FF1FA60BFF1F2309FF1F3409FF1FF1
:10283000490AFF1F300DFF1FF0B587B00EAD2F788E
:102840000FAD2D780593AC46634614000E4D0CAACF
:1028500012782E7803930D9B009201932200059B22
:10286000029701F0DDF92E70012C01D0042C08D163
:10287000802206498B889343054A1278D20113437C
:102880008B8007B0F0BDC0461C09FF1F6C11FF1FF5
:102890007809FF1F0B001B3B70B504003020E02BB4
:1028A0000DD81300E025493BFF3B9BB2ED00AB4246
:1028B00005D8034B200019825A8201F071F970BDCE
:1028C0008410FF1F10B501F01BFB054B00205B6857
:1028D000052B04D9034A5268D20200D4980810BDCF
:1028E00000100040FCE100E070B501F011FA0D4B62
:1028F0001B68FC33DC691D6AFFF7E4FF641984423E
:1029000004D2094B01241B68002B07D004220024A9
:10291000064B1A70064A93690133936101F080FBFC
:10292000200070BDAC64FF1F9809FF1F2309FF1F23
:10293000FC0FFF1F70B50C4D2B68FC335C6A01F077
:10294000E7F9FFF7BFFF2B680025FC339B6AE3180C
:10295000834204D2054B1B68AB4200D1051B01F03A
:102960005FFB280070BDC046AC64FF1F9809FF1FC5
:10297000D722044B92009B5810B5002B00D09847EB
:1029800010BDC0460000FF1F10B501F0DBF8FFF7D7
:10299000EFFF2749274BCA6D274C1A4084235B0061
:1029A0001343CB65254B1B68186A01F041F9244B92
:1029B000244A1A60244B254A1A60A022244B520054
:1029C0001A60244B187801F0FBFA2000224901F02C
:1029D0003FFB0023A3600233A360204B2049236008
:1029E00003232048A36001F033FB10221E4BFF207D
:1029F0001A60802252031A60802292031A60802299
:102A000012041A6001F0ECF9012001F0C1FAFA2079
:102A1000400001F01DFA582001F0F2FA134801F0CD
:102A200027F9012001F0CCF9072001F0F1F810BDE1
:102A300000F0004000FEFEFF14100040AC64FF1FD9
:102A4000000003400180063DBC0003403408000044
:102A5000A40003404A0AFF1F71020000C3090000DE
:102A6000FFFF3F002810004000E100E0307500004B
:102A7000674E336888331B6883F3088801F068F970
:102A8000644A6549136800200B401360634B644A35
:102A90001B68934200D1A6E001F0E2F90221614AED
:102AA00013688B431360FFF76FFF5F4B5F4C187821
:102AB000C0B201F0C5FA0023A3600233A3605C4BEF
:102AC0000120236001F0B4F80323A36001F068FA49
:102AD000040001F015FA050001F062FA554B186088
:102AE00001F0CEFA544B1968621A531EA14200D26B
:102AF00013008022D203934201D39B029B0A3268C7
:102B0000D16AC90700D471E04C491C0C09689BB21A
:102B10004C4359432402090A641803264849FC32ED
:102B200093680A6847489B1A474A076812684749EA
:102B30009B18474A9A1833409208DB190A600360D1
:102B4000042B03D9013233400A6003600E68414907
:102B5000A619300001F0ECF93F4F3E493B68C3181D
:102B60003B603000019301F0ABF83C4E3068081830
:102B700038493060884205D9019B01333B6001F040
:102B80009FF8316001F044FA354B1B78002B0DD0D3
:102B900001F0B6F9334B621B196812188A4232D21F
:102BA0004919091B091A304801F052FA2F4E337A9D
:102BB000002B0ED001F0A4F9621BF16812189142AB
:102BC00024D94919091B091A294801F041FA00239F
:102BD0003372284B83F3088801F00AF9002001F0D2
:102BE0003FF901F045FA01F03BF95CE7DC0199009F
:102BF0000234641A5900641A09214B438033CB40D4
:102C0000A408E41889E7FA218900CCE71A49DBE730
:102C1000AC64FF1F1CF00040FFFFC1FF0C0AFF1F48
:102C2000B641210310000040490AFF1F1410004064
:102C3000C3090000100AFF1F340AFF1F380AFF1FD4
:102C4000200AFF1F280AFF1F1C0AFF1F240AFF1F5C
:102C5000C4090000710200006008FF1F2C0AFF1F5A
:102C60001C09FF1FE408FF1F00100040740BFF1F2A
:102C70003C10004000000020DC050000A022054BB5
:102C800092009B5810B5002B01D0984710BD00F062
:102C900097FFFBE70000FF1FA122054B92009B5806
:102CA00010B5002B01D0984710BD00F089FFFBE75D
:102CB0000000FF1FA222054B92009B5810B5002B6D
:102CC00001D0984710BD00F07BFFFBE70000FF1F1D
:102CD000A322054B92009B5810B5002B01D09847BA
:102CE00010BD00F06DFFFBE70000FF1FA422054BA5
:102CF00092009B5810B5002B01D0984710BD00F0F2
:102D00005FFFFBE70000FF1F70B501F0F9F84F4BC4
:102D1000186001F04DF80400C30702D401F068F90F
:102D200070BD00224A4B1A604A4B187801380428BB
:102D300029D800F01FFF0320181C2400200001F0F8
:102D400067F80128ECD0444C2378042B6ED100F0B6
:102D500057FF0028E4D001F09BF9582001F050F90A
:102D600002232370DCE7200000F0B2FFE9E7200037
:102D700001F0EEF8E5E7200001F092F8E1E720002D
:102D800001F0F6F8DDE701F083F80500012808D12D
:102D9000324B1B78053B012B03D82000FFF76EFF59
:102DA000D1E72D4B1B78022B01D0052B20D1022D12
:102DB00028D12B4B9B7BAB431CD12000FFF76CFF32
:102DC000264B18780128BED16405BCD4244925229D
:102DD0004B7B034205D1233A13405A4253412633D9
:102DE0001A000B7D9342AED9322001F049F8AAE7D0
:102DF000022D07D1194B1B78052B11D12000FFF7AD
:102E000059FFDDE7012D0BD1012B03D12000FFF786
:102E10005FFF98E7062B03D12000FFF767FF92E7DB
:102E2000200000F0CDFE022D8DD1C9E7032B04D187
:102E30000C4B987C00F064FF72E7072B00D06FE723
:102E4000094B987B00F0ACFF6AE7C0469C09FF1F66
:102E50009809FF1F9009FF1F2309FF1F1C09FF1F6F
:102E6000A60BFF1FBC0BFF1FD40BFF1FFA210A4B41
:102E70000A4A49001A640A4A5A500A4A04395A50FE
:102E8000094A08319A64094A5A50094A5C315A5031
:102E9000084ADA667047C0460000FF1F3928FF1F46
:102EA0003529FF1FE928FF1F1924FF1FA927FF1F2E
:102EB000B91EFF1F8D1EFF1FF7B50B0CFF27012248
:102EC000009300233C001E001D009446019089B22F
:102ED00062469A401000084018413618B6B2FF2FDB
:102EE00002D1012E00D19FB2009802401A41AD18C4
:102EF000ADB2FF2C02D1012D00D19CB20133102BB9
:102F0000E6D10320012E07D1012D04D1019B24011C
:102F1000E4191C700138FEBD102EFCD10238102DB2
:102F2000F9D00230F7E700008023F7B59C46264B26
:102F3000264F01932649274A274D284C284B022823
:102F40001AD1604638600868264E30408026360325
:102F50003043086001990978002909D11660224A96
:102F60002A60224A2260E02219689143A03A1BE0BD
:102F70008021C9021160F2E766463E600F68194E73
:102F80003E408027FF023E430E60019909780029E8
:102F90000DD1176001280ED1154A2A60154A22600A
:102FA000E02219689143C03A0A431A60F7BD8021B4
:102FB00089021160EEE7E0210F4A02432A600F4ABE
:102FC00022601A688A43F0E74B0AFF1FE0000340C3
:102FD000D80003409000034000000340500003402D
:102FE00040000340FFFFE3FF0280063D80450822CA
:102FF0000180063D806608220080069880550822E0
:10300000F8B51E4B80261A68002014003440324266
:1030100032D11A681A4F32431A6001223B680630D7
:1030200093433B6000F004FE0122164D2B681E43C3
:103030002E603B680A2613433B608027BF00124B7B
:103040001B683B4211D1013EF6B2FF2E09D17E2210
:103050000E4B1C682B68E40B1440934323432B60F6
:1030600005E0082000F0E4FDE9E7002EEFD1802222
:103070002B68600893432B60F8BDC046C4F0004045
:103080005CF0004018F0004068F0004060F0004044
:1030900010B500F0ADFD01215820034A00F028FFD3
:1030A000FFF7AEFF10BDC046600AFF1F10B57822C3
:1030B0000021034800F0D4FF00F0DAFE002010BD2C
:1030C000A067FF1F70B5040000F022FE00230C2053
:1030D0000B4A010059438D18515C00290DD0A142C3
:1030E00008D1012300246B7000F01AFF00F098FF54
:1030F000200070BD01330A2BEBD11224F6E7C04645
:10310000A067FF1F70B5040000F002FE0023190045
:103110001D000D4A1078002806D0A0420CD1557031
:1031200001310C320A29F5D1002B0AD100F0A0FEA2
:1031300000F076FF002070BD5078461EB0411B188D
:10314000EEE700F0EDFEF3E7A067FF1FF7B5040020
:103150000C20002384460E4D019267465F43E85DD4
:103160007E19A04212D000280BD10A4B9C46624621
:103170001B7808331370019B70707C557160B360CD
:10318000FEBD01330A2BE8D10320F9E70720F7E75A
:10319000A067FF1F9C67FF1F8020F8B5484BC00544
:1031A0001B68C1248360474BFF251A680123134322
:1031B0004361454BA4001A68444B40211A60444BBC
:1031C0001A68444B1A60444B1A59AA431A51C52233
:1031D00092009E58AE433143802699509F583F49F4
:1031E000F6010F403E439E509E5880273602360A15
:1031F0003043985080201A5900020A4002431A5165
:1032000004341A59364E3F04324080263A431A514C
:103210001A5936061202120A32431A5108341A5940
:1032200080260A4002431A51C32292009F58B44696
:10323000AF4337439F509F58294E0F4007439F503D
:103240009F58374080263604374380269F509F582A
:1032500036063F023F0A37439F50C0221F59AF43F3
:103260003A431A511A591202120A1643C6221E5123
:1032700092009C58AC4365462C439C509C580025BA
:103280000C4020439850C72080001A58154C11401C
:10329000C02212020A431A50134B1B78DB08AB42C0
:1032A00001DC0020F8BD2378002B06D0A368002B9A
:1032B00000D0984701350C34EEE71220F2E7C04603
:1032C000AC43FF1FA843FF1FB0F000409867FF1FEB
:1032D000B4F000409467FF1F00E100E0FF00FFFF33
:1032E000FFFF00FFA067FF1F9C67FF1F030010B5D3
:1032F0001F2809D8072200201340072404490A7810
:10330000A24313430B7010BD00230620F5E7C0460F
:103310009C67FF1F034A0449136800200B40136099
:103320007047C0461CF00040FFFFC1FF054B064937
:103330001B780A6805485B0702401B0B13430020FB
:103340000B6070479C67FF1F1CF00040FFFFC1FF30
:1033500070B50C25FFF7EAFF0A4B1C780A4BE4080E
:103360006543ED18002C01D1200070BD2B78002B97
:1033700006D06B68002B00D09847013C0C3DF1E76C
:103380001220F2E79C67FF1F9467FF1F1FB5002103
:1033900002220B0001910091052000F019FC02238C
:1033A0000B490A681A42FCD120230393039B5A1E3F
:1033B0000392002BFAD1074A1368002BFCDA0B2486
:1033C0006C442000012100F0DBFD207804B010BD2A
:1033D00090C8004000C8004013B504000A4B019398
:1033E000019B002B01D1112016BDFFF7CFFF230059
:1033F0000340044205D0052000F01AFC019B013B6C
:10340000EDE71800F0E7C046FFFFFF0707B500F043
:103410007FFC80220821D205936A0191002B01D103
:103420000739916202210C4A11600199481E0190EE
:103430000029FAD103311160053101910199481E2B
:1034400001900029FAD11160002B02D18022D2050F
:10345000936200F0E5FD07BD00C00040F0B52D4CC3
:1034600089B02378002B4FD1FEF7A8FA02232A4F08
:1034700003903A681A42FCD120230693069B5A1EF9
:103480000692002BFAD1254E3368002BFCDA01207E
:10349000FFF7A2FF011E02D0112009B0F0BD03000A
:1034A00003220190009005AD9F2000F091FB0321C5
:1034B000280000F065FD02233A681A42FCD120235F
:1034C0000793079B5A1E0792002BFAD13368002BF3
:1034D000FCDA0120FFF780FF0028DDD10398FEF71A
:1034E00081FAAA786B7811041B020B4329780B43ED
:1034F00063601300113B0A49052B07D80123934051
:10350000A3600B60012323700020C6E780231B0308
:10351000F6E7C0469443FF1F90C8004000C8004033
:103520009808FF1F1E4B30B55A6818781D4B85B0A0
:10353000D31859424B4101210093002300F038FD7C
:10354000194B1A4A02259A6300221A6510325A65ED
:103550008022C4219D65164B1648D202DA67890085
:103560004258154B80241A4080231B0413434350B8
:10357000642341200393E40500F006FA402000F0A4
:1035800003FA6562039D6B1E0393002DFAD103239A
:103590006362FFF73BFFA562FFF760FF05B030BD38
:1035A000A043FF1F95FFFEF700C80040050001FF84
:1035B00004E100E000E100E0FFFF00FFF0B585B0AE
:1035C0000700FEF7FBF9022305002D4C22681A4282
:1035D000FCD120230093009B5A1E0092002BFAD1AD
:1035E000284E3368002BFCDA0120FFF7F5FE002897
:1035F00003D01124200005B0F0BD234B236002232B
:1036000022681A42FCD120230193019B5A1E019289
:10361000002BFAD13368002BFCDA0120FFF7DCFE27
:103620000028E6D1194B1F60022322681A42FCD100
:1036300020230293029B5A1E0292002BFAD1336878
:10364000002BFCDA0120FFF7C7FE0028D1D1104B78
:103650002360022322681A42FCD120230393039B98
:103660005A1E0392002BFAD13368002BFCDA01209A
:10367000FFF7B2FE041EBCD12800FEF7B3F9B9E78C
:1036800090C8004000C8004001000006A8C80040E3
:103690000180000110B50020FFF790FF10BD000071
:1036A00010B5064B18705960FFF73CFF002113203E
:1036B000034AFFF74BFD002010BDC046A043FF1F8B
:1036C0002535FF1FF0B5040085B003920291FEF787
:1036D00075F9882263035B0B52051A438023DB05CF
:1036E0009D6A8023274F0092BA68002601901B0331
:1036F0009A420CD9F82326001B041E401C4206D017
:103700008022214B52025E6219680A431A60002D22
:103710000BD100F0FDFA02221C4B1A608023DB055E
:103720005A62013A9A6200F07BFC0023039A9342AA
:1037300020D1002D0AD100F0EBFA144B03221D60BA
:103740008023DB055A629D6200F06AFC8023BA6820
:103750001B039A4208D9002E06D000220A4B0C49BE
:103760005A621A680A401A600198FEF73BF9002075
:1037700005B0F0BD009A0299D2181278CA540133EC
:10378000D4E7C0469443FF1F00C8004000C000407B
:10379000FFFFFEFFF0B587B0029103920400FEF731
:1037A0000DF9019000F0B4FA802302250122234E86
:1037B000DB0535605D629A6200F032FC204F3B68A9
:1037C0002B42FCD120230493049B5A1E0492002B0D
:1037D000FAD11C4D2B68002BFCDA0120FFF7FCFD11
:1037E000002802D0112007B0F0BD2000039A0299F2
:1037F00000F06EFB022304003A681A42FCD1202339
:103800000593059B5A1E0592002BFAD12B68002BBD
:10381000FCDA0120FFF7E0FD051EE3D100F078FAA5
:1038200080230322DB0535605A629D6200F0F8FBBD
:103830000198FEF7D7F8E0B2D5E7C04600C00040D7
:1038400090C8004000C80040F0B5802489B0060050
:10385000FEF7B4F8E405A36A02250393029000F092
:1038600057FA0123304F3D606562A36200F0D8FB38
:103870002E4C23682B42FCD120230593059B5A1E16
:103880000592002BFAD12A4D2B68002BFCDA01207F
:10389000FFF7A2FD002803D01124200009B0F0BDDD
:1038A000244B2360022322681A42FCD12023069372
:1038B000069B5A1E0692002BFAD12B68002BFCDACD
:1038C0000120FFF789FD021EE6D11B4B03211E607C
:1038D000030001900090202000F07AF90223226872
:1038E0001A42FCD120230793079B5A1E0792002BF4
:1038F000FAD12B68002BFCDA0320FFF76DFD041EC4
:10390000CAD100F005FA80230322DB053C605A622D
:103910009C6200F085FB039B002B01D1FFF776FD35
:103920000298FEF75FF8B8E700C0004090C800407A
:1039300000C800400100000694C8004007B500021E
:1039400001910422000A01A9FFF724FF0EBD000027
:1039500073B5050005240B4AA3005B429B18196848
:103960006B46DE1D3000FFF7A7FA022804D133783A
:103970002B55013CEFD276BD052CFCD00128FAD1A5
:103980000230F8E7140900111F2807D8012380220C
:103990008340D20591680B43936070473F2808D855
:1039A0000123802220388340D20551690B435361A3
:1039B000F3E75F28F1D80123802240388340D20505
:1039C000116A0B431362E8E71F2807D80122802100
:1039D0008240C9058B6893438B6070473F2808D8A5
:1039E0000122802120388240C9054B6993434B61F5
:1039F000F3E75F28F1D80122802140388240C905D1
:103A00000B6A93430B62E8E71F2810D8802302005B
:103A1000DB05153A1968012A06D82022914319605E
:103A200019680A431A60704701228240F6E73F286E
:103A300011D880230200DB05353AD968032A06D85D
:103A400010229143D960D9680A43DA60EBE701227A
:103A500020388240F5E75F28E5D842238022181AF3
:103A6000413B8340D205516A99435162516A0B43ED
:103A70005362D8E710B50400012813D1A0221849D9
:103A800092050B685B015B0913430B60154B164AEB
:103A900019681140154A0A431A60402219680A43FE
:103AA0001A6010BD0028FCD101000A2000F040F986
:103AB00021000B2000F03CF9C0220A4B920019684B
:103AC0000A4340211A601A688A431A60B0220449E6
:103AD00012060B685B015B0913430B60E1E7C0460C
:103AE00014F000401CF000407F00FEFF80FD01004C
:103AF00072B6074A1368013313600422054B1A603B
:103B00000023054A13608022D2055360FEE7C046B9
:103B10007808FF1FC0F00040C4F0004005490B6862
:103B2000002B05D1044A0A6004490A60044A136064
:103B30007047C046140AFF1F841E0000380AFF1F8A
:103B4000C4F000400023034A1360034A1360034A91
:103B50001360704754F0004040F1004044F10040D1
:103B600002B4714649084900095649008E4402BC16
:103B70007047C04602B4714649084900095C4900D3
:103B80008E4402BC7047C04603B4714649084000E9
:103B90004900095A49008E4403BC704700000000E8
:103BA00001B40248844601BC604700BF116E0000AA
:103BB00001B40248844601BC604700BF8D8200000A
:103BC00001B40248844601BC604700BFE917010008
:103BD00001B40248844601BC604700BF496D010042
:103BE00001B40248844601BC604700BF6D0B010070
:103BF00001B40248844601BC604700BFED68010083
:103C000001B40248844601BC604700BF01D70000F0
:103C100001B40248844601BC604700BFF90D0100B1
:103C200001B40248844601BC604700BF9D6A0000A1
:103C300001B40248844601BC604700BF018900000E
:103C400001B40248844601BC604700BF0D52010028
:103C500001B40248844601BC604700BF53B900006C
:103C600001B40248844601BC604700BF51B800005F
:103C700001B40248844601BC604700BF8D110100B9
:103C800001B40248844601BC604700BFA1AF0000F8
:103C900001B40248844601BC604700BFA9D80000B7
:103CA00001B40248844601BC604700BF8B5201004A
:103CB00001B40248844601BC604700BFBD5C0100FE
:103CC00001B40248844601BC604700BF090E0000F1
:103CD00001B40248844601BC604700BF09340100BA
:103CE00001B40248844601BC604700BF19FA0000D5
:103CF00001B40248844601BC604700BFD9B000004F
:103D000001B40248844601BC604700BF4DF9000081
:103D100001B40248844601BC604700BF75A9000099
:103D200001B40248844601BC604700BF75F800003A
:103D300001B40248844601BC604700BF89A300115A
:103D400001B40248844601BC604700BFDD3F00006B
:103D500001B40248844601BC604700BFC9A9000005
:103D600001B40248844601BC604700BFC115010090
:103D700001B40248844601BC604700BFCD0C01007D
:103D800001B40248844601BC604700BFD1AE0000C8
:103D900001B40248844601BC604700BF5976010067
:103DA00001B40248844601BC604700BFC1F700006F
:103DB00001B40248844601BC604700BFBD0B01004E
:103DC00001B40248844601BC604700BFE51201000F
:103DD00001B40248844601BC604700BF85C10000B1
:103DE00001B40248844601BC604700BFED6B01008E
:103DF00001B40248844601BC604700BF79970000C7
:103E000001B40248844601BC604700BF71B00000A5
:103E100001B40248844601BC604700BF0134010080
:103E200001B40248844601BC604700BF89370100E5
:103E300001B40248844601BC604700BFB352010090
:103E400001B40248844601BC604700BFE9D40000C9
:103E500001B40248844601BC604700BF85120100DE
:103E600001B40248844601BC604700BF016C0100F8
:103E700001B40248844601BC604700BFADAE0000FB
:103E800001B40248844601BC604700BF61370100AD
:103E900001B40248844601BC604700BFDD0C01004C
:103EA00001B40248844601BC604700BFF5350100FB
:103EB00001B40248844601BC604700BFF9ED000030
:103EC00001B40248844601BC604700BFC1A50000A0
:103ED00001B40248844601BC604700BF95730100ED
:103EE00001B40248844601BC604700BFE90B0100F1
:103EF00001B40248844601BC604700BF016701006D
:103F000001B40248844601BC604700BFC95C01009F
:103F100001B40248844601BC604700BFE94C01007F
:103F200001B40248844601BC604700BF21A90000DB
:103F300001B40248844601BC604700BF090E00007E
:103F400001B40248844601BC604700BF89440000B8
:103F500001B40248844601BC604700BF053401003B
:103F600001B40248844601BC604700BFE9F6000086
:103F700001B40248844601BC604700BFF935010026
:103F800001B40248844601BC604700BF3D71010096
:103F900001B40248844601BC604700BF69110100BA
:103FA00001B40248844601BC604700BF156B0100A4
:103FB00001B40248844601BC604700BFC56D0100E2
:103FC00001B40248844601BC604700BFEDA5000073
:103FD00001B40248844601BC604700BFCD4C0100DB
:103FE00001B40248844601BC604700BF0DB7001110
:103FF00001B40248844601BC604700BFDD0A0100ED
:1040000001B40248844601BC604700BF7912010038
:1040100001B40248844601BC604700BFD54401009A
:1040200001B40248844601BC604700BF9DA900005E
:1040300001B40248844601BC604700BFE927000084
:1040400001B40248844601BC604700BF89140100E6
:1040500001B40248844601BC604700BF2D6C0100DA
:1040600001B40248844601BC604700BFB70E00009F
:1040700001B40248844601BC604700BF855201007C
:1040800001B40248844601BC604700BFC16601001C
:1040900001B40248844601BC604700BF6DF60000D1
:1040A00001B40248844601BC604700BF21440000BF
:1040B00002000000DABF001101000000D0BD0011B5
:1040C00002000000D6BF001101000000F040FF1FF9
:1040D00002000000D8BD0011010000002862FF1F8F
:1040E00002000000D4BF0011030000009C61FF1F0C
:1040F0001200000002000000DABF00110100000001
:1041000018BE001102000000D6BF0011010000001F
:1041100015BE00110200000022BE001103000000C5
:10412000D761FF1F02000000D4BF00110300000090
:10413000EC61FF1F02000000D6BF0011010000006B
:1041400014BE00110200000020BE00110300000098
:10415000AD61FF1F02000000D4BF0011030000008A
:10416000CE61FF1F02000000DABF00110100000055
:1041700058BE001102000000D6BF0011010000006F
:104180003942FF1F020000006ABE0011010000005A
:1041900053BE001102000000D6BF00110100000054
:1041A0003842FF1F0200000068BE0011010000003D
:1041B000F461FF1F02000000D6BF001101000000E3
:1041C0003742FF1F0200000066BE00110100000020
:1041D00043BE001102000000D6BF00110100000024
:1041E0003642FF1F0200000064BE00110100000003
:1041F0003EBE001102000000D6BF00110100000009
:104200003542FF1F0200000062BE001101000000E5
:1042100039BE001102000000D6BF001101000000ED
:104220003442FF1F0200000060BE001101000000C8
:1042300034BE00110202020202020000000000006F
:104240000D0C0000D54C00119B4C0011C8BE001194
:1042500090011D0018001800FFFF0701020304056C
:10426000060201060000000000000000000000003F
:10427000000000000000000000000000000000003E
:104280000300000002000000DABF0011010000007E
:10429000E8BE001102000000D6BF001101000000BE
:1042A000F442FF1F02000000F2BE001101000000F6
:1042B0002262FF1F02000000D4BF001103000000B3
:1042C0008C64FF1F02000000D6BF00110100000037
:1042D000F442FF1F02000000F0BE001101000000C8
:1042E0002462FF1F02000000D4BF00110300000081
:1042F0008464FF1F126C6C6C0000000000580040CA
:10430000151600000001000000000111FFFF000071
:104310005048593600000000000000000B00050066
:10432000F0000000B4000028002800283075A0002C
:10433000A000A000A00000080008E001F0001000AC
:10434000100010001000100010005000500050002D
:1043500010001000D0070000000000000F00010056
:104360000500307507001000010081FF000000000B
:10437000FF000000717500117973001109710011BF
:10438000FFFF0100FF0000008D9F0011099D00113B
:10439000219C001100000000000000000000080047
:1043A000040000003B0001085902E00188212800B8
:1043B000FF00000002000000DABF00110100000051
:1043C000A0C0001102000000D6BF001101000000D3
:1043D0003144FF1F02000000D2BF001101000000A5
:1043E0005868FF1F02000000D6BF00110100000046
:1043F0003044FF1F02000000D0BF00110100000088
:104400002E44FF1F02000000D6BF00110100000073
:104410002C44FF1F02000000CEBF0011010000006D
:104420002444FF1F180018001D0090010200000323
:104430000202000002000000DABF001101000000CB
:10444000B4C0001102000000D6BF0011010000003E
:104450007444FF1F02000000CCBF001100000000E8
:104460000000000002000000D4BF001103000000A3
:064470007868FF1F20FF29
:040000051FFF184180
:00000001FF
